:100000000C94D4020C94F1020C94F1020C94F102C1
:100010000C94992F0C94F1020C94F1020C94F102BF
:100020000C94F1020C94F1020C9436280C94F227F3
:100030000C9432290C94F1020C94F1020C94F1020C
:100040000C94F1020C94F1020C94F1020C94F10264
:100050000C94F1020C940E290C94F1020C94F10210
:100060000C94F1020C94F1020C94F1020C94F10244
:100070000C94F1020C94F1020C94F1020C94F10234
:100080000C94F1020C94F1020C94F1020C94F10224
:100090000C94F1020C94F1020C94F1020C94F10214
:1000A0000C94F1020C94F1020C94F1020501090286
:1000B000A10185020901A1000509190129081500FE
:1000C0002501950875018102050109300931158165
:1000D000257F95027508810609381581257F9501D0
:1000E00075088106050C0A38021581257F95017572
:1000F000088106C0C005010980A101850319012AF4
:10010000B700150126B700950175108100C0050CD8
:100110000901A101850419012AA002150126A002E6
:10012000950175108100C00660FF0961A101096297
:10013000150026FF00952075088102096315002629
:10014000FF00952075089102C005010906A101056F
:100150000719E029E7150025019508750181029529
:1001600001750881010507190029FF150026FF0008
:100170009506750881000508190129051500250156
:10018000950575019102950175039101C00000006C
:10019000000000000000000000000000000000005F
:1001A000000000000000000000000000000000004F
:1001B000007E0F00D4FFFFFFC700000078000000A2
:1001C00000000000002A2B280000000000000000B2
:1001D000000000000000000029000000002C1E3478
:1001E00020212224342627252E362D3738271E1F7E
:1001F000202122232425263333362E37381F0405A9
:10020000060708090A0B0C0D0E0F10111213141516
:10021000161718191A1B1C1D2F3130232D350405F4
:10022000060708090A0B0C0D0E0F101112131415F6
:10023000161718191A1B1C1D2F3130354C000101DF
:100240000101010101010102020202020202020295
:100250000303030303030303040404040404040565
:100260000505050506060606060707070707080829
:100270000808090909090A0A0A0B0B0B0C0C0C0DDA
:100280000D0D0E0E0E0F0F0F101011111112121373
:10029000131414151516161717181819191A1A1BEE
:1002A0001B1C1D1D1E1E1F2020212222232424254D
:1002B0002626272829292A2B2C2D2D2E2F30313286
:1002C00032333435363738393A3B3C3D3E3F404196
:1002D00042434445464748494A4C4D4E4F5051537E
:1002E00054555658595A5B5D5E5F61626465666835
:1002F000696B6C6D6F7072737577787A7B7D7E80B9
:1003000082838587888A8C8E8F91939596989A9C04
:100310009EA0A2A3A5A7A9ABADAFB1B3B5B7BABC18
:10032000BEC0C2C4C6C9CBCDCFD1D4D6D8DBDDDFE9
:10033000E2E4E7E9EBEEF0F3F5F8FAFDFFE3003570
:100340000014001A000800150017004B00E000041C
:10035000001600070009000A000000E2001D001B53
:100360000006001900050000000000000000004C1D
:10037000422A22294130002F00130012000C0018DD
:10038000001C004E00343133000F000E000D000B36
:100390000000003134380037003600100011000032
:1003A000000000000000002B422C32284101002DEB
:1003B000023A003B003C003D003E00010057001E99
:1003C000021F02200221022202000067001E001FFD
:1003D0000020002100220000000000000000002397
:1003E000520100010045004400430042004100402A
:1003F000003F0001005600270226022502240223A6
:100400000200000100270026002500240023000030
:1004100000000000000000235201000100A800536A
:100420000054005F00600061005600A9006700559D
:10043000005C005D005E0057000000010062005992
:10044000005A005B00850000000000000000000171
:1004500000010023524D0039004700480046004A81
:10046000000100AA00653149004F00520050000110
:1004700000000001000100010051004D00010000DA
:1004800000000000000000010001002352010001F3
:10049000000100010001000100010001002078239B
:1004A000782578277829780100000021782478269B
:1004B0007828782A78010000000000000000000180
:1004C0000001000100010001000100D200DE00D1A6
:1004D00000D900010001000100D000CD00CF00DAFA
:1004E00000000001000100DF00CE00DD000100007F
:1004F0000000000000000001000100010009025B93
:1005000000030100A0FA0904000001030101000931
:10051000211101000122440007058103080001099F
:100520000401000203000000092111010001222240
:1005300000070582032000010705030320000109CD
:100540000402000103000000092111010001227BC7
:1005500000070584032000011201000200000008CA
:10056000EDFE0000010001020001160341006E00D3
:10057000670065006C00570069006E00670073003B
:100580000000200344006F007200790061006E00DB
:10059000200061006E00640020004E004D0031001C
:1005A000370000000403090411241FBECFEFDAE076
:1005B000DEBFCDBF25E0AEE8B2E001C01D92A63798
:1005C000B207E1F712E0A0E0B1E0EEEDF5E602C01F
:1005D00005900D92AE38B107D9F70E9459290C94B5
:1005E00065320C940000982FE091660540912D052E
:1005F00057E0E41302C080E008952E2F30E05E9FA4
:10060000F0011124E25DFA4F8181681306C08081F8
:10061000981303C085818111EFCFF9013196E770FE
:10062000E8CFFC01AC014C5F5F4F8FEF91E321916C
:10063000822728E030E087FF09C0880F89272150F2
:100640003109C9F7E417F50791F70895880FF7CF37
:10065000E8EDF0E080818E7F80831092E2001092BE
:10066000DA001092E100A0EEB0E08C9181608C93F2
:1006700080818F77808319BCA7EDB0E08C918E7F4D
:100680008C9380818F7E808310921605089520912F
:10069000E4003091E50095E6A9012091EC00822F5D
:1006A000817020FF06C08091E80080FF06C080E0D6
:1006B00008952091E80022FD1AC080912305882327
:1006C00089F0853089F08091EB0085FD0FC0209185
:1006D000E4003091E50042175307F9F29150E1F63A
:1006E00084E0089582E0089583E0089581E008950C
:1006F0008091250587FF13C08091E80082FF06C026
:100700008091E8008B778093E80004C080912305F6
:100710008111F2CF0895809123058823D9F3809128
:10072000E80080FFF8CF8091E8008E77ECCF982F1B
:100730009093E900242F762F50E0891731F07091C3
:10074000EC002091ED005091F00021FD07C09F5F6B
:10075000973071F78093E90081E008953091EB00C4
:100760003E7F3093EB003091ED003D7F3093ED0004
:100770003091EB0031603093EB007093EC002093EC
:10078000ED005093F0002091EE0027FDE0CF80E0D7
:100790000895B0E0A0E0EFECF3E00C94C030C8EDB9
:1007A000D0E088818F7E8883E7EDF0E080818160F2
:1007B000808384E082BF81E08093160588818E7FEC
:1007C000888302EE10E0F80110821092DA0081EEC8
:1007D000C82ED12CF601108288818F77888388817A
:1007E0008068888388818F7D888319BC1092230557
:1007F00010922405109222051092210590EEE92E08
:10080000F12CF70180818B7F8083888181608883D0
:1008100042E060E080E00E949703F60180818E7FD5
:100820008083F801808181608083808188608083FB
:10083000F70180818E7F8083888180618883CDB736
:10084000DEB7E8E00C94DC30FC01CB0120912B05F5
:1008500030912C052617370790F0009729F4209146
:10086000E8002E772093E80040E0009751F4411112
:1008700008C08091E80082FF31C080E00895C9017E
:10088000F3CF209123052223A9F12530A9F120914E
:10089000E80023FD2DC02091E80022FDEACF209141
:1008A000E80020FFE2CF3091F3002091F2000097A2
:1008B00019F02830310558F041E02830310509F0B1
:1008C00040E02091E8002E772093E800CECF4191C0
:1008D0004093F10001972F5F3F4FE9CF80912305AF
:1008E000882341F0853041F08091E80083FFC1CF3B
:1008F00081E0089582E0089583E00895089580914D
:100900001805089587E797E79093010880930008FA
:1009100088E19AE00FB6F894A895809360000FBE26
:1009200090936000FFCF9C014FB7F894809112051F
:1009300090911305A0911405B09115054FBF821B2E
:10094000930B0895A4E0B0E0E8EAF4E00C94C6301C
:100950008FB7F8942091120530911305409114053A
:100960005091150529833A834B835C838FBF69813E
:100970007A818B819C812496E2E00C94E2302FB73F
:10098000F8948091120590911305A0911405B091EF
:1009900015052FBF08959C01FC0132968FEF90E062
:1009A0004191461751F08F3F19F4411101C0892F31
:1009B0009F5F9630A9F78F3F09F40895280F311DE6
:1009C00087FD3A95F90162830895A3E0B0E0EBEE6C
:1009D000F4E00C94C6309C0180910F0590911005B5
:1009E00082179307A1F03093100520930F05E09133
:1009F0000D05F0910E05309751F084E089833B831B
:100A00002A830084F185E02DCE0101960995239675
:100A1000E2E00C94E230A3E0B0E0E1E1F5E00C9418
:100A2000C6309C0180910B0590910C0582179307AD
:100A3000A1F030930C0520930B05E0910D05F0918A
:100A40000E05309751F083E089833B832A8300842D
:100A5000F185E02DCE01019609952396E2E00C94F4
:100A6000E23080910905882359F0E0910D05F0915D
:100A70000E05309729F00190F081E02D0995089539
:100A800080E008950E94BF0420910505309106057D
:100A9000232B21F0809301059093020520910705F7
:100AA00030910805232B21F08093FF0490930005DB
:100AB000E0910D05F0910E05309749F082E08093AA
:100AC00003050680F781E02D83E095E00995089500
:100AD0008091FE0480FD16C081FD16C082FD16C007
:100AE0008091FD048823A1F0883280F428E0829F61
:100AF000C001112468E270E00E940131862F672B4B
:100B000039F0089582E0089584E0089588E008951A
:100B100081E008958091FE0480FD14C081FD14C021
:100B200082FD16C08091FC04882381F08E3180F410
:100B300020E5829FC00111246EE170E00E94013126
:100B4000862F089584E1089588E2089588E0089545
:100B500080E50895282F35EB2303C001112497FF6A
:100B600004C080589109892F089580589F4FFBCF6A
:100B7000FA01882311F009950895FB01FCCFFC01CF
:100B800080910A05811123C0E731F1051CF17797A7
:100B9000CF01880F991FDC01AE0FBF1FA45CBB4FB4
:100BA00011963C911197361307C03C91341304C041
:100BB00012963C91321771F031E030933B04E80F0C
:100BC000F91FE45CFB4F61834083228303C0E7315C
:100BD000F105F4F2089510923B040895EBE6F5E078
:100BE00024813AE0231B08F420E0248380913A0416
:100BF000816080933A040895EBE6F5E024813AE0C1
:100C0000230F08F42FEF248380913A0481608093AE
:100C10003A040895922F20916B05237071F0809310
:100C20006C0560936D05433808F042E840936E050B
:100C300020913A04292B20933A040895EBE6F5E03D
:100C4000438128E0421B08F440E0818121E0628179
:100C500090E00E940A060895EBE6F5E0438128E063
:100C6000420F08F44FEF818121E0628190E00E9401
:100C70000A060895EBE6F5E0628128E0621B08F4BD
:100C800060E0818121E0438190E00E940A0608959E
:100C9000EBE6F5E0628128E0620F08F46FEF8181F6
:100CA00021E0438190E00E940A060895EBE6F5E01A
:100CB000818121E0438162818850990B0E940A065C
:100CC0000895EBE6F5E0818190E021E043816281C7
:100CD00008960E940A060895262F90916B0593703E
:100CE00061F081110BC0946090936B0510923301F9
:100CF00060913A04622B60933A040895813210F0B7
:100D00009068F2CF880F880F982BEECF90916B05EB
:100D1000969596958FEF890F913009F480E261E006
:100D20000E946C06089580916B05869586958F5F6D
:100D3000813208F081E061E00E946C0608959DE038
:100D4000899F802D1124980F913408F090E4209110
:100D50000A05222321F0983128F097E10895873180
:100D600008F487E10895E42FF0E0EE0FFF1FE3534E
:100D7000FE4F9081921B97FD9195292F38E1239F7B
:100D8000212D1124620F08950F931F93522F10E00D
:100D9000F801EE0FFF1FE353FE4F9081905797FD30
:100DA0009195000F111FF801EB56FE4F01AD005257
:100DB000110B50039001519F300D112408E310E0F6
:100DC000091B110997FD13954003F001419FF00D98
:100DD0001124E20FF31F9F01220F331F2E0F3F1F1D
:100DE00037FF02C021583F4F220F232F221F330B02
:100DF000620F1F910F9108950F931F93522F10E0D0
:100E0000F801EE0FFF1FEB56FE4FA1ADA052BB0B3A
:100E10009D015203F001539FF00D1124000F111F8B
:100E2000D801A353BE4F0C910057110B4003900102
:100E3000419F300D11242E0F3F1F37FF02C0215C50
:100E40003F4F96E0359527959A95E1F7620F1F91F0
:100E50000F9108950F931F93522F10E0F801EE0F9A
:100E6000FF1FEB56FE4FA1ADA052BB0B9D015203DD
:100E7000F001539FF00D1124000F111FD801A3534F
:100E8000BE4F0C910057110B40039001419F300D54
:100E900011242E0F3F1F37FF02C021583F4F220F52
:100EA000232F221F330B620F1F910F910895EF9292
:100EB0000F93972F23E0029FB0011124759567953A
:100EC0006E0D792F0F91EF900895322F50E0FA01B7
:100ED000EE0FFF1FEB56FE4F91AD905297FD91958F
:100EE000440F551FFA01E353FE4F2081231B330BA0
:100EF000290F311D97FD3A95620F0895E42FF0E018
:100F0000EE0FFF1FEB56FE4F61AD621B0895E42FFD
:100F1000F0E0EE0FFF1FE353FE4F6081621B089568
:100F2000622F0895582FA22FE42FF0E0EE0FFF1F3D
:100F3000E353FE4F208134EE239F212D112490E0B6
:100F400030E0245E3F4F2A1B310937FF03C0319543
:100F50002195310943E0220F331F4A95E1F7821BA7
:100F6000930B97FD80E0282F259F212D1124822FA0
:100F700008951F93172F922FE42FF0E0EE0FFF1F1D
:100F8000E353FE4F208134EE239F212D1124472F60
:100F900050E030E0245E3F4F291B310937FF03C08A
:100FA00031952195310993E0220F331F9A95E1F78E
:100FB000421B530B57FD40E0742F719F712D11247C
:100FC0001F9108950E94BF050895FF920F931F93EC
:100FD000CF93DF93182F062FF42ED0E0C0E02F2DF3
:100FE000402F612FCE010E94E2072196C034D10527
:100FF000B1F7CDB7DEB7E5E00C94DF30FC019B0123
:10100000009729F480E077FF2BC080E80895AC01B9
:1010100097FF04C044275527481B590BB901640F9B
:10102000751F37FD10C0241B350BC901A5E0880FC3
:10103000991FAA95E1F70E94013180E2861BF7FF14
:101040000FC081950895CB0165E0880F991F6A95BF
:10105000E1F7BA01621B730B0E94013180E6EECF0B
:101060000895EF920F93CF93DF93D72FC82FBA0134
:10107000C9010E190E94FE07602F681B7D2F8C2F5F
:10108000DF91CF910F91EF9008950F93CF93DF935E
:10109000D72FC82FBA01C9010E94FE07682F600F21
:1010A0007D2F8C2FDF91CF910F910895EF920F93A9
:1010B0001F93CF93DF93D62FC72F182FBA01C901E3
:1010C0000E19010F0E94FE07081B019F012D11241C
:1010D0006D2F7C2F802FDF91CF911F910F91EF907B
:1010E0000895EF920F931F93CF93DF93D62F172F6F
:1010F000C82FBA01C9010E19010F0E94FE07702FF7
:10110000781B719F712D11246D2F8C2FDF91CF9142
:101110001F910F91EF9008950F931F93CF93DF933B
:10112000D62FC72F182FBA01C901212F201B022F3C
:101130000E94FE07982F990F990F282F291B200F27
:10114000219F212D11246D2F7C2F822FDF91CF9194
:101150001F910F9108950F931F93CF93DF93D62F75
:10116000172FC82FBA01C901212F201B022F0E945F
:10117000FE07982F990F990F782F791B700F719F89
:10118000712D11246D2F8C2FDF91CF911F910F9115
:101190000895982FE82F96FDE0952E2F2F7096FD3D
:1011A0002F5FE695E695E695E670F0E0E258FE4F93
:1011B0008181829F802D212D112482958F7022950F
:1011C000207F822B2081820F97FD81958058089582
:1011D0000F931F93CF93DF938B01D82FC42F822FB0
:1011E0000E94C908EC2FF0E0EE0FFF1FE353FE4F03
:1011F00090819058980F97FD9195990F692F2CE049
:10120000629F612D1124600F712F8D2FDF91CF917F
:101210001F910F91089540912F015091300125E0C9
:1012200038E0429FC001439F900D529F900D1124C2
:10123000875E994C9093300180932F01890F089518
:101240009C018230910508F408959FEF213E8EE1C4
:10125000380740F4C90145E0969587954A95E1F72E
:1012600098E0980F61E0E62FE90FFF27FF1FAF011D
:1012700055954795842F449FF001459FF00DF00D43
:1012800011242E173F0738F49FEF940F961758F745
:101290008FEF860F08954F3FE9F361E0640FF6CFBB
:1012A0000F93CF93DF93D72FC82FF90147FD4195B7
:1012B00028E330E0241B310947FD3395229FA0012C
:1012C000239F500D500D1124EE9FC001EF9F900DF4
:1012D000900D1124840F951F0E942009982F990FBB
:1012E000692F680F600F7D2F8C2FDF91CF910F91A9
:1012F00008959C0190E080E0269F812D369F800D0F
:10130000911D11240895A4E0B0E0E9E8F9E00C94FF
:10131000C63020916F0530E1230F08F42FEF60E114
:10132000822F90E00E947909BC0188EB9BE00E942B
:10133000ED30B0E0A0E0CD012496E2E00C94E23084
:10134000982F80910A05882329F081E0973128F0B1
:1013500080E003C081E09034D8F70895B0E0A0E0C9
:10136000E4EBF9E00C94BE30262F472FE82FF0E095
:10137000E35CFD4F711109C06491862FE62F7E2F2B
:10138000CDB7DEB7EAE00C94DA30E72EF12CE49129
:1013900086E0689F80011124CFEFD0E0C801BE0134
:1013A0000E94ED30DB0130E0220F331F55E5569FE0
:1013B000C001579F900D1124281B390B622F660F17
:1013C000260FCE018E199F09E89F6001E99FD00C7E
:1013D00011246D2D429FA0011124452F5527CE01C8
:1013E000841B950BE89FA001E99F500D1124852FC8
:1013F0005E01A21AB108AE9C9001AF9C300DBE9C5C
:10140000300D1124232F3327C21BD30BEC9F9001E7
:10141000ED9F300D1124A330B105B1F00C3F93E0E6
:10142000190760F4A130B10599F01297A9F00F3FA8
:10143000110508F0A4CF8D2D632FA1CFA430B105E5
:1014400071F01697C1F39BCF652F8E2FED2D97CF9F
:101450006E2FE52F8D2D93CF832F6E2FF7CF8E2FED
:10146000E32F8DCFB0E0A0E0E8E3FAE00C94C130C8
:10147000EC01FC01E35BFD4F8081682349F1D090D2
:101480006D0500916E0510916C05E12EF12C0E9406
:101490000B09282FC7018C549F4F68E671E00E940A
:1014A00001318E199F0997FD03969595879595951E
:1014B00087952370612F289F600D11247D2D802F2B
:1014C0000E94AE09462F672F282FCE010E94E20707
:1014D000CDB7DEB7E7E00C94DD30EF92FF920F93CB
:1014E0001F93CF93DF937C01809135010E949F066B
:1014F000C82F192F60916F056695669521E0620FE0
:1015000008F46FEF80916705909168050E94790952
:10151000082FD0E0C11740F0812F0E94A009CDB75D
:10152000DEB7E6E00C94DE30FE01E35BFD4F808128
:1015300090913601892391F060916C0570916D0551
:1015400080916E05202F4C2FF70109950E94AE095E
:10155000462F672F282FCE010E94E2072196DACF6F
:10156000A4E0B0E0E6EBFAE00C94C0306C018091AE
:1015700035010E949F068B83F92E60916F05669559
:10158000669580916705909168050E947909182FEA
:1015900080E4810F0E94C90880588983812F0E94AE
:1015A000C90880588A839B81892F90E09C838B8314
:1015B0009B819F1538F08F2D0E94A0092496E8E0AA
:1015C0000C94DC30EB81FC81E35BFD4F80819091DA
:1015D00036018923A9F060916C0570916D058091A9
:1015E0006E05E12E0B812A814981F60109950E9441
:1015F000AE09462F672F282F8B819C810E94E2071E
:101600008B819C810196D2CFB0E0A0E0EAE0FBE0C4
:101610000C94BA303C01809135010E949F06C82F7E
:10162000192F60916F056695809167059091680507
:101630000E947909F82ED0E0CE01880F991F9C01F5
:101640002B563E4F6901C11740F0812F0E94A0091F
:10165000CDB7DEB7EEE00C94D630FE01E35BFD4F74
:10166000808190913601892379F1F60180AD282F90
:101670002057330B590181ADE82FE052FF0B4F018A
:10168000AA9C9001AB9C300D300D1124EE9FC0013F
:10169000EF9F900D900D1124820F931F0E9420093F
:1016A000082F60916C0570916D0580916E05EF2C8F
:1016B0009401A501F30109950E94AE09462F672FF9
:1016C000282FCE010E94E207F2E0CF0ED11C219616
:1016D000BACFAF92BF92DF92EF92FF920F931F9318
:1016E000CF93DF935C01809135010E949F06C82F44
:1016F000192F60916F056695809167059091680537
:101700000E947909D82ED0E0CE01880F991F9C0144
:101710002B563E4F7901C11768F0812F0E94A00916
:10172000DF91CF911F910F91FF90EF90DF90BF90CD
:10173000AF900895FE01E35BFD4F808190913601EB
:101740008923C1F0F70121AD2052330B40AD405742
:10175000550B60916C0570916D0580916E050D2D96
:10176000F50109950E94AE09462F672F282FCE015B
:101770000E94E207F2E0EF0EF11C2196CCCF1F93FE
:10178000CF93DF93EC01FC01E35BFD4F8081682385
:10179000B1F00E940B09182F0E940B0920E8829FCC
:1017A000C00111247FE7790F612F80916E050E949F
:1017B000AE09462F672F282FCE010E94E207DF9146
:1017C000CF911F91089580E00895F894E82FE29555
:1017D000EF70F0E041A18F7021E030E0B90102C06C
:1017E000660F771F8A95E2F7CB01962F9095942389
:1017F00091A392A1892B82A378940895A4E0B0E0EC
:10180000E4E0FCE00C94C63080910905882371F077
:101810000E94A20469837A838B839C8369817A8185
:101820008B819C812496E2E00C94E2300E94A20419
:1018300069837A838B839C838091F1029091F20279
:10184000A091F302B091F40229813A814B815C812D
:10185000280F391F4A1F5B1F29833A834B835C8300
:10186000DDCF9091010392FF10C041E0282F247139
:10187000243009F040E031E0282F2871283009F0A9
:1018800030E0431711F02CE0822793FF10C041E0B5
:10189000282F2471243109F040E031E0282F2871ED
:1018A000283109F030E0431711F02CE08227309105
:1018B000020330FF10C051E0282F2171213009F0C0
:1018C00050E041E0282F2871283009F040E05417FB
:1018D00011F029E0822731FF10C041E0282F21714B
:1018E000213109F040E031E0282F2871283109F03A
:1018F00030E0431711F029E0822794FD877E089598
:10190000803E9105C1F1C8F48133910509F47DC091
:1019100048F48932910509F46DC08A32910509F4C1
:101920007BC0089589339105D1F082389105B9F0D3
:101930008533910509F459C00895843E9105C1F19C
:1019400038F4823E910521F1833E910531F10895ED
:10195000863E9105C1F1873E9105E1F10895209100
:101960000103237009F065C02091020323FF14C016
:1019700089E290E008952091010320FD43C0309159
:10198000020330FF09C024FF4EC090E080E00895BC
:101990002091010322FDF7CF08952091010322FD3C
:1019A00045C03091020330FD44C024FFF5CFEDCF98
:1019B0002091020321FFF0CF8091010384FDE5CF48
:1019C00087EE90E008952091010323FFE5CF24FDE9
:1019D000DCCFF6CF2091010323FD2EC0309102030E
:1019E00031FFE3CF84EE90E008952091010325FFBD
:1019F000D3CFBECF2091010325FD21C0209102034A
:101A000023FFCACF89E390E0C7CF2091010326FFCF
:101A1000C3CF8AE290E008952091010326FFBCCF56
:101A200081E390E0089583EE90E0089582EE90E0E7
:101A3000089580EE90E0089586EE90E0089585E3A5
:101A400090E008951F93CF93DF930E94800CEC01E8
:101A50008115924508F05FC0C11580E5D80708F0F0
:101A6000DDC0C03ED10538F5CD3CD10508F0AEC093
:101A7000C83AD10580F4C53AD10508F0A4C0C130F8
:101A8000D10509F443C0CE010497813A9105F0F1E4
:101A9000D0E0C0E03BC0CE01885A91094B97C0F717
:101AA000C85AD0E0CC0FDD1FC55CDE4F0990D8814D
:101AB000C02DD4642BC0C11590E4D907F0F4C11532
:101AC00020E2D20708F0C4C0C83ED105F8F0CE012C
:101AD0009A9581159F41E0F68D2F0E94310C182FA9
:101AE000CE0199270E94800CC12FD0E0DC2FCC279B
:101AF000CC27DF71C82BD92B09C0CE0199270E94B2
:101B0000800CCC27DF70C82BD92BD06ACE01DF9197
:101B1000CF911F910895C03882E5D807B8F5C03637
:101B200092E5D90708F05BC0C03422E5D207C8F4BB
:101B3000C03282E5D80708F04BC02C2F2695269599
:101B400090E2299F900111248C2F8370C1E0D0E096
:101B500002C0CC0FDD1F8A95E2F7C22BD32BDD68C4
:101B6000D5CF2C2F26952695277080E2289F9001AF
:101B700011248C2F8370C1E0D0E002C0CC0FDD1F98
:101B80008A95E2F7C22BD32BDC68C0CFC03C92E52C
:101B9000D90760F48C2F8F71C03AD245A8F5C82FB1
:101BA000D0E0DC2FCC27C46FD06AB0CFCE01805CF0
:101BB0009245809708F06CCFDC2FCC27CC27DF71C3
:101BC000C06FD06AA3CFA497D064A0CFD0659ECFBA
:101BD000CF71D0E0DC2FCC27C16FD06A97CF2C2FEC
:101BE00026952695277080E2289F900111248C2F3E
:101BF0008370C1E0D0E002C0CC0FDD1F8A95E2F710
:101C0000C22BD32BDA6882CF0E94310CC82FD0E0D0
:101C1000DC2FCC27CC27DF71D06278CF8C2F8F714F
:101C20000E94310C55E0D695C7955A95E1F7CF70D3
:101C3000D0E0DC2FCC27282F30E084FF05C044E023
:101C4000220F331F4A95E1F7C22BD32BD0695ECF09
:101C50008D2F8F710E94310C182FCE0199270E9471
:101C6000800CC12FD0E0DC2FCC27CC27DF71C82B14
:101C7000D92BD2CF982F90958091C1028923809340
:101C8000C10208958091660590912D05981301C0B9
:101C900008958F5F8770FACF292F983078F58730B5
:101CA00068F590E037E0239F800D911D1124682F87
:101CB000677023E0969587952A95E1F7FC01EE0F72
:101CC000FF1FE80FF91FE656FD4F50E040E080E0AF
:101CD000219130E0062E02C0369527950A94E2F74E
:101CE00021703327042E01C0220F0A94EAF7822BB9
:101CF0004F5F5F4F4330510559F7089580E00895D5
:101D0000292F983090F5873080F590E037E0239FB9
:101D1000800D911D1124282F277041E001C0440F30
:101D20002A95EAF723E0969587952A95E1F7FC0135
:101D3000EE0FFF1FE80FF91FE656FD4F90E080E021
:101D400070E05191DF0111979B01082E02C036957A
:101D500027950A94E2F7217021952527242325272A
:101D60002C9301968330910561F7089580930003C9
:101D700008959091000321E030E0F90101C0EE0FD9
:101D80008A95EAF7D90102C0AA0FBB1F6A95E2F74C
:101D9000EA2B01C0220F4A95EAF7892F8E23E81318
:101DA00005C0292B822F0E94B60E08952095292365
:101DB000F9CF21E030E001C0220F8A95EAF72095A3
:101DC0008091000382230E94B60E08959091B6027E
:101DD000809589238093B602282F277069F489178C
:101DE00059F09091020392FF07C0869586958695DB
:101DF0000E94D90E1092B602089521E030E001C091
:101E0000220F8A95EAF780910003822B0E94B60E7A
:101E100008958093FF02089540910505909107056C
:101E200020910805662309F469C0942B922B209118
:101E30000605922B31F098E09093FC0491E090938A
:101E4000FD048D3C41F40E948A058195809306052E
:101E50000E94420508958E3C19F40E948A05F6CF2F
:101E60008F3C31F40E948A05819580930505F0CF5F
:101E7000803D19F40E948A05F8CF893D29F40E941B
:101E8000680580930705E4CF8A3D21F40E94680528
:101E90008195F7CF8B3D31F40E9468058195809341
:101EA0000805D6CF8C3D19F40E946805F8CF9FE253
:101EB000980F983070F4815D990B21E030E001C0FB
:101EC000220F8A95EAF780910405822B80930405FE
:101ED000BFCF8D3D31F48091FE0481608093FE047C
:101EE000B7CF8E3D21F48091FE048260F7CF8F3D05
:101EF00009F0AECF8091FE048460F0CF8D3C59F4A0
:101F00008091060587FF0DC01092060541110BC098
:101F10001092FC0408C08E3C81F4809106051816CE
:101F20009CF3442381F08091070590910805892B4B
:101F300009F08ECF1092FD048BCF8F3C49F447FF00
:101F4000F0CF10920505809106058111ECCFE0CF0E
:101F5000803D19F41416ACF3E4CF893D29F4191629
:101F600004F710920705DDCF8A3D19F497FFD9CF0A
:101F7000F8CF8B3D29F427FFD4CF10920805D1CF9D
:101F80008C3D19F41216CCF3CCCF9FE2980F983009
:101F900090F4815D990B21E030E0B90102C0660F39
:101FA000771F8A95E2F7CB018095909104058923EC
:101FB00080930405B6CF8D3D31F48091FE048E7F71
:101FC0008093FE04AECF8E3D21F48091FE048D7F80
:101FD000F7CF8F3D09F0A5CF8091FE048B7FF0CF26
:101FE0000F931F93CF93DF938B01EA019091230509
:101FF000943061F58093E9008FEF9091E800815073
:1020000095FD06C095ED9A95F1F700008111F5CF89
:102010008091E80085FF1AC00E944703811111C01A
:102020008091E80085FD06C08091E8008E7780935E
:10203000E800F2CFF80181918F018093F1002197A0
:1020400079F78091E8008E778093E800DF91CF9157
:102050001F910F910895BC0143E050E084E00E947D
:10206000F00F0895BC0146E050E084E00E94F00FBC
:102070000895CF93DF93D82FC92F48E050E0682F01
:10208000792F81E00E94F00F88E0ED2FFC2FA9E16D
:10209000B5E001900D928A95E1F7DF91CF91089517
:1020A00080913B04882341F1529A3BB13B7F2BB195
:1020B00024604FB7F8948CE394E0FC0101965081C2
:1020C00068E02BB9000000C057FF3BB9550F000076
:1020D00000C000C000C03BB900C06A9591F754E051
:1020E0008C3F950751F74FBF8FE594E00197F1F7CB
:1020F00000C0000010923B040895B0E0A0E0E3E8C7
:10210000F0E10C94BE30F82EE92ED62EC72E8A01AF
:102110008091F002AA24A394B12C8A3018F48AE0AA
:10212000A82EB12CC1E0D0E06D2D7C2D8F2D9E2DE1
:10213000F8010995811104C02196AC16BD062CF456
:10214000CDB7DEB7EAE00C94DA30CC9F9001CD9F9A
:10215000300D300D112490E080E045E34A95F1F711
:102160000000019682179307C1F7DECFCF93C82FE7
:102170006FEF811164E285E290E00E94DE316FEF43
:10218000C11164E086E290E00E94DE316FEFC11180
:1021900067E287E290E00E94DE31CF910895CF930D
:1021A000DF93C9EED1E060E0CE010E94DE312196DE
:1021B000C11584E0D807B9F7DF91CF9108951F9337
:1021C000CF93DF93962F122F632F8430D8F498305B
:1021D000C8F44730B8F4C42FD0E0CC0FDD1F2EE098
:1021E000929FC00DD11D112490E7899FC00DD11D74
:1021F0001124CE0189960E94DE31612FCE018A968C
:102200000E94DE31DF91CF911F910895AF92BF926E
:10221000CF92DF92FF920F931F93CF93DF93B12C56
:10222000A12C00E0650110E013C0FE01259134915E
:102230004F2D612F802F0E94DF102296F39487E0AC
:10224000F812F3CF87E0C80ED11C1F5F183039F0A9
:10225000E601CC0FDD1FC35CDC4FF12CE6CF0F5F36
:1022600088E3A80EB11C0430E9F6DF91CF911F91ED
:102270000F91FF90DF90CF90BF90AF90089580E0D6
:102280000E94B61060E088E290E00E94DE310E9479
:1022900006110E94CF1081E00E94B610089585E2D9
:1022A00090E00E94C031843289F486E290E00E947E
:1022B000C031843059F487E290E00E94C03191E04F
:1022C000873209F090E0892F8170089580E0FCCF7B
:1022D0000F931F93CF93DF93843030F5683020F550
:1022E000473010F5C42FD0E0CC0FDD1F2EE0629FE9
:1022F000C00DD11D112430E7839FC00DD11D1124C5
:10230000CE0189960E94C031082F10E0102F0027BF
:10231000CE018A960E94C0319801282BC901DF9115
:10232000CF911F910F91089590E080E0F8CF462F54
:10233000672F783038F4473028F4843018F40E943E
:102340006811089580E090E00895B0E0A0E0EBEA25
:10235000F1E10C94C1307C01009100038091FF02F7
:10236000082BC3E0D0E010E0DC2EC8010C2E02C028
:10237000959587950A94E2F780FD09C02197A0F70B
:10238000D12C8D2DCDB7DEB7E7E00C94DD30B70151
:102390008C2F0E9497110E94220D019779F3F1CFA3
:1023A000CF93DF93D82FC92F0E94A5116D2F7C2FBB
:1023B0000E9497110E94220DDF91CF910895FC0198
:1023C00084818823A1F0808191810E94D011282FDF
:1023D00092959F70963091F060F4925F9F7092306A
:1023E00030F481E0203F81F030F4283E30F080E08E
:1023F00004C09A5FF3CF243FD1F7089581E0283ECF
:1024000020F0213FA1F7F9CF08950895A6E0B0E0AC
:10241000ECE0F2E10C94C53049835A83392F89816D
:102420009A81332399F0222389F00E94A511182F55
:10243000682F89819A810E94800E69817A81812F1B
:102440000E9497112696E3E00C94E1300E944C0E16
:10245000182FF3CF48E050E068E170E08BE695E09C
:102460000E94CE3110923A040895A6E0B0E0EBE36A
:10247000F2E10C94B9300E94FE0B60931503709347
:102480001603809317039093180320916B05322F46
:1024900033703D83332321F0422F469546954D837B
:1024A00030913301323009F4F8C580F4311115C090
:1024B00010923501609367057093680580936905F4
:1024C00090936A0581E08093330103C0333009F4AF
:1024D000EEC52696EFE00C94D530809132015D81F7
:1024E000581322C023704091310150E081E024173D
:1024F000150609F480E081708093370180917005A2
:1025000090913601981739F08093360140E060E0F1
:1025100080E00E94E5076D81613260F4E62FF0E013
:10252000E959FD4C0C94153181E0E5CF80913701DC
:10253000811102C080E031C140E060E080E00E9493
:10254000E507F8CF809135010E949F06082F9983F7
:1025500060916C0570916D0580916E050E94AE09C9
:10256000F62EE72ED82E10E07981071720F0872F5E
:102570000E94A00912C1F801E35BFD4F8081909198
:102580003601892331F02D2D4F2D6E2DC8010E946B
:10259000E2070F5F1F4FE8CF809135010E949F0631
:1025A000082FD92EF0906D0510916E0580916C0565
:1025B0008983682F7F2D812F0E94AE09C62EB72EEA
:1025C000A82E60916F059981690F7F2D812F0E9440
:1025D000AE096983F72EE82E10E00D1510F08D2D51
:1025E000C7CFF801E35BFD4F80812091360128239E
:1025F00059F02E2D49816F2D80FD03C02A2D4C2DC1
:102600006B2DC8010E94E2070F5F1F4FE6CF80913C
:1026100035010E949F069983E0906D05D0906E056C
:1026200020916F0530E4F32E3F2D329F312D112480
:10263000F32E082F10E04981041710F0842F98CF53
:10264000F801E35BFD4F8081909136018923B9F059
:10265000F801EE0FFF1FEB56FE4F81AD82958F7094
:1026600060916C058F9D600D11247E2D8D2D0E9433
:10267000AE09462F672F282FC8010E94E2070F5F7F
:102680001F4FD9CF809135010E949F069983E0901A
:102690006D05D0906E0520916F0590E4F92E5F2DA9
:1026A000529F512D1124F52E082F10E06981061735
:1026B00010F0862F5DCFF801E35BFD4F8081909194
:1026C00036018923D9F0F801EE0FFF1FEB56FE4FBC
:1026D00060ADF69EB001112485E0759567958A95E9
:1026E000E1F780916C05680F7E2D8D2D0E94AE095B
:1026F000462F672F282FC8010E94E2070F5F1F4F48
:10270000D5CF809135010E949F06082F9983F090C4
:102710006C0510916D05E0906E0560916F056695F2
:102720006695669580916705909168050E94790984
:102730000E94C90820E8280F27FD2195220F7E2D31
:10274000279F212D11246F2D712F822F0E94AE09FA
:10275000F62EE72ED82E10E08981081708F008CF52
:10276000F801E35BFD4F808190913601892331F0C0
:102770002D2D4F2D6E2DC8010E94E2070F5F1F4FB8
:10278000EBCF89EB97E00E946D0A07C082E997E0E2
:10279000FACF8BEA98E00E94690B9091350121E015
:1027A000290F20933501811173C482E08093330196
:1027B0008091370181116CC48D81882309F475C41F
:1027C000892F0E949F0685CE8CE898E0E4CF81E7B0
:1027D00098E00E94040BE1CF86E598E0FACF80E90B
:1027E00097E0D1CF87E897E0CECF8EE797E0CBCFC9
:1027F00085E697E0C8CF87E597E0EBCF80E599E0E5
:10280000CACF85E498E0C7CF81E398E0E2CF8AE2BF
:1028100097E00E94B00AC1CF8CEF96E0FACF84EC2B
:1028200096E0F7CF809135010E949F0699839091A1
:102830003701911120C060916F0520E1620F08F40B
:102840006FEF80916705909168050E9479096AE0B1
:1028500070E00E94ED30892B61F40E940B09A0E426
:102860008A9FC001112460913601892F90E00E9457
:10287000320A89817DCE082F10E0B981EB2EF12C30
:102880000E151F05B4F760913601C8010E94320A87
:102890000F5F1F4FF5CF809135010E949F069983EE
:1028A0009091370191111FC060916F0520E1620F77
:1028B00008F46FEF80916705909168050E9479098F
:1028C00065E070E00E94ED30892B99F60E940B09BB
:1028D000E0E48E9FC001112460913601892F90E0C1
:1028E0000E94BF0BC6CF082F10E0F981EF2EF12C0C
:1028F0000E151F050CF0BDCF60913601C8010E9476
:10290000BF0B0F5F1F4FF4CF809135010E949F06D0
:10291000082F9983E0906D05F0906E0510916C057D
:1029200060916F05669566956695809167059091B3
:1029300068050E9479090E94C90820E8280F27FD30
:102940002195220F3CE0239F212D1124612F620F3E
:102950007E2D8F2D0E94AE09F62EE72ED82E10E088
:102960002981021710F0822F03CEF801E35BFD4F9F
:10297000808190913601892331F02D2D4F2D6E2DC0
:10298000C8010E94E2070F5F1F4FEACF88EE98E070
:10299000FACE83EB96E0F7CE809135010E949F0638
:1029A000F92E409167055091680560916905709115
:1029B0006A058091190390911A03A0911B03B091AD
:1029C0001C0384179507A607B70708F04FC00E949D
:1029D0000B0930E4839F80011124012F1127F80196
:1029E000E35BFD4F808190913601892309F43EC05D
:1029F0000E940B0981FD3CC00E940B0989830E9443
:102A00000B0940E8849FC00111247FE7790F809172
:102A10006E0569810E94AE09462F672F282FC801D5
:102A20000E94E20720916F0530E1230F08F42FEF99
:102A300060E1822F90E00E947909BC0184EF91E06F
:102A40000E94ED308091670590916805A09169051D
:102A5000B0916A05860F971FA11DB11D80931903C0
:102A600090931A03A0931B03B0931C038F2D80CD6A
:102A700080E070E01982CDCF4091DD035091DE03FC
:102A80006091DF037091E003809167059091680584
:102A9000A0916905B0916A0584179507A607B70745
:102AA00008F448CD80913701811150C080913501E3
:102AB0000E949F069E83E82EF12C53E0859F8001A3
:102AC0001124035E1C4F2E81E21608F47CC0822F75
:102AD0000E94A009811138C020E04E814150550B61
:102AE0007A01822F90E08E159F050CF481C00E9420
:102AF0000B098701000F111F81FF92C00E0D1F1DD2
:102B0000F801E35EFC4F1082118212820E94830959
:102B100069837A838B839C83809167059091680594
:102B2000A0916905B0916A0529813A814B815C8148
:102B3000820F931FA41FB51F8093DD039093DE03C4
:102B4000A093DF03B093E0038E8112CD40E060E0FC
:102B500080E00E94E507FDE1EF2EF3E0FF2E10E09C
:102B600000E00E940B0981FF10C0D7011C92119652
:102B70001C92119712961C920F5F1F4FB3E0EB0E41
:102B8000F11C0034110569F791CF0E940B0989836C
:102B90000E940B09B0E88B9FC00111247FE7790FD9
:102BA000C801880F991F800F911FFC01E35EFC4F45
:102BB0006F01698180916E050E94AE09D6016D9307
:102BC0007D938C93D9CFF701E35BFD4F808190918A
:102BD0003601892339F0F801228140816181C701E2
:102BE0000E94E2070D5F1F4FFFEFEF1AFF0A6BCF46
:102BF000AC01440F551F480F591F435E5C4F0196AF
:102C0000FC01EE0FFF1FE80FF91FE35EFC4F808110
:102C10009181A281FA0180839183A2832F5F61CF8A
:102C20000E940B09D82E0E940B09F0E88F9FC0016B
:102C300011247FE7790F0E0D1F1D035E1C4F6D2DB4
:102C400080916E050E94AE09D8016D937D938C939F
:102C50005DCF80913701882329F040E060E080E07B
:102C60000E94E507809135010E949F06592E4091F0
:102C70006705509168056091690570916A058091BA
:102C8000F9039091FA03A091FB03B091FC03841720
:102C90009507A607B70708F084C060916C0570918E
:102CA0006D0580916E050E94AE096E83772E682EA9
:102CB00041EEE42E43E0F42E05E911E0580148010D
:102CC0006701F2E0F98302C031E03983D6012D912A
:102CD0006D01F40181914F0190E0222309F463C05A
:102CE000262D4E81672D0E94E207D50116968C9104
:102CF000262D4E81672D90E00E94E207D6018C912F
:102D0000F60131978083B1E0AB1AB108E981E13077
:102D1000D9F6D80112968C9190E0F70122812223F6
:102D200009F44CC0262D4E81672D0E94E207D80180
:102D300014968C91262D4E81672D90E00E94E2071B
:102D40000E940B09837091E009F090E0D701129680
:102D50009C93B3E0EB0EF11C095F1F4FE1E00D3CCB
:102D60001E0709F0ABCF0E94830969837A838B83A6
:102D70009C838091670590916805A0916905B09149
:102D80006A0529813A814B815C81820F931FA41FC0
:102D9000B51F8093F9039093FA03A093FB03B093BC
:102DA000FC03852DE5CB20E040E060E00E94E207D7
:102DB000F501868120E040E060E09DCF20E040E02A
:102DC00060E00E94E207F801848120E040E060E0DA
:102DD000B4CF809135010E949F06982EC92E809114
:102DE0003701882361F040E060E080E00E94E50761
:102DF000E2E0F4E088E3DF011D928A95E9F7809133
:102E00003501811117C08091FE039091FF030E944C
:102E100093049C0181E02931310508F480E080931E
:102E2000FD032931310530F00E94BF049093FF0368
:102E30008093FE03B12CA12CD12C97E0792E25E5AF
:102E4000622E3AEA832E5524539405C0FCE0FA150D
:102E500008F457C0D12C2D2D30E07B9C800111242B
:102E6000F801EB56FE4FE20FF31FE080E91408F47F
:102E700040C0EC1408F03DC0A394F12CF701E35BD3
:102E8000FD4F808190913601892309F432C00E5F95
:102E90001B4F020F131FF801F081F9834F2F262DCE
:102EA000421B08F440E070916D05382D5F2F350FFF
:102EB00008F43FEF50916E05232F220F230F2E5F52
:102EC000259F212D1124682D641B822F0E94AE099D
:102ED000462F672F282FC7010E94E2078091FD032C
:102EE000882339F02981652D261B08F420E0D801BC
:102EF0002C93D394B7E0DB12AECFB394E8E0BE12CC
:102F0000A5CF8C2D35CB20916E05298333E0239FEF
:102F1000800111241695079516950795502EA22E1F
:102F2000B12C8FEF90E0B5010E940131762E809197
:102F30003701882371F040E060E080E00E94E507FF
:102F4000E2E0F4E088E3DF011D928A95E9F7109250
:102F50000104809100048F5F80930004F12CE12C28
:102F6000A01AB10A6701612CD701AE5FBB4F4D01BA
:102F700080910104862909F046C00E948A31853576
:102F800095400CF040C02981F4012083F601EB56F6
:102F9000FE4FE081EF3FD1F0D601AE5FBB4F2C91E9
:102FA000F0E0521608F041C030E0201B310B209FAA
:102FB000C001219F900D309F900D1124B5010E94FA
:102FC000ED30262F4981CF010E94E207639457E03C
:102FD000C50ED11C68E06612CBCF7FEFE71AF70A67
:102FE00087E0E816F10409F0BDCF80910004781263
:102FF00002C010920004809101048F5F8D3100F5B2
:103000008093010497CAF601EE5FFB4F808188230D
:1030100009F4BCCF3981831708F0B8CF9091000430
:103020007912B4CF81508083B1CF4981429FC001D2
:103030001124B8010E94ED30462F20E060E0C3CF9C
:10304000109201042CE234E087E049E054E09981D9
:103050009150A2E0B4E0F901873049F4D1966C9127
:10306000D1977981761303C0D1969C93D1976081D3
:103070007981671710F090837783119631964A17FC
:103080005B0751F78150275031098111E2CF52CAB5
:10309000AD81AA2309F41DCA93CBBD81B09332013F
:1030A0002370209331010E94501083E00CCA80915C
:1030B0003A0481110E942A12C0906705D0906805D9
:1030C000E0906905F0906A05809109058823B9F0C0
:1030D0002FB7F8948091120590911305A0911405D3
:1030E000B09115052FBF8C199D09AE09BF094097F6
:1030F000A105B10508F4EDC910923301EAC90E9497
:10310000FE0BDC01CB01EFCF9091020392FB222753
:1031100020F9281779F080FB92F9909302036091CF
:1031200001037091020384E090E00E94FC3182E090
:103130000E94E60E08958091C1029091B802892BF9
:103140009091B702992389F0892B90E022E932E02F
:10315000F90140812F5F3F4F41119F5F42E02839C5
:103160003407B1F791111092B7028093900248E0B2
:1031700050E069EB72E080E992E00E949A31892B7D
:10318000A9F088E0E0E9F2E0A9EBB2E001900D924D
:103190008A95E1F7E0910D05F0910E05309731F039
:1031A0000280F381E02D80E992E009950895CF93A4
:1031B0001092C102C6E0E2E9F2E0DF018C2F1D921D
:1031C0008A95E9F790E080E00E940B0590E080E0AE
:1031D0000E94E5041092B8020E949B18E3E0F5E01B
:1031E000DF011D92CA95E9F71092FC041092FD04CC
:1031F0001092FE040E944205CF910895AAE2B0E029
:10320000E4E0F9E10C94C53085E295E0FC0101961B
:103210002091F100208325E08D329207B9F780914B
:103220002605893009F456C0C8F4823009F4B3C0C9
:10323000833009F482C0813071F18091E80083FF0E
:1032400085C280912505909126059A3008F07EC2AE
:10325000E92FF0E0E857FD4C0C9415318A3009F461
:1032600089C08B3051F780912505813231F78091EB
:10327000290590912A05892B01F78091E800877F25
:103280008093E8000E9478038091270580933401A1
:103290000E94D718D2CF80912505813A71F680918E
:1032A000E800877F8093E8008091290590912A05A6
:1032B000892B61F468E089E195E070E00E942404C4
:1032C0008091E8008B778093E800B7CF60E090E0D2
:1032D00080E0F3CF80912505813209F0AECF809157
:1032E000290590912A058D7F892B09F0A6CF809121
:1032F000E800877F8093E8008091E80082FF18C093
:103300009091F3008091F200029731F48091F100E6
:10331000813011F0863021F48091F10080931805FE
:103320008091E8008B778093E8000E94780385CF36
:10333000809123058111E0CF80CF80912505813ACE
:1033400009F07BCF8091290590912A05892B09F0FE
:1033500074CF8091E800877F8093E8008091E80037
:1033600080FFFCCF809134018093F1008091E800D0
:103370008E77D9CF80912505813209F05ECF80917B
:10338000E800877F8093E8000E94780380912805F9
:103390008093170552CF80912505813A09F04DCFD2
:1033A0008091E800877F8093E8008091E80080FFAB
:1033B000FCCF80911705D8CF803899F0823809F07A
:1033C000C5C1809129058F70873008F0BFC18093F7
:1033D000E9008091EB0085FB882780F91092E900D5
:1033E00006C08091210590912205911182609091F3
:1033F000E800977F9093E8008093F1001092F1002D
:103400008091E8008E779EC1882309F48CC18230B8
:1034100009F09CC18091270581118FC180912905F8
:103420008F702FEF280F263008F090C18093E900AD
:103430002091EB0020FF81C1933031F48091EB00AB
:1034400080628093EB0079C19091EB009061909342
:10345000EB0021E030E001C0220F8A95EAF72093CB
:10346000EA001092EA008091EB008860EACF8111B7
:103470006DC1109127051F778091E3008078812B23
:103480008093E3008091E800877F8093E8000E94AA
:1034900078038091E80080FFFCCF8091E300806892
:1034A0008093E30082E0111183E0809323054EC1F5
:1034B0008058823008F04AC1409127055091280574
:1034C0004C3D83E05807A1F583E08A838AE2898333
:1034D0004FB7F894DE01139620E03EE051E2E32F6F
:1034E000F0E050935700E49120FF03C0E295EF70A5
:1034F0003F5FEF708E2F90E0EA30C0F0C7968D935B
:103500009D932F5F243159F74FBF8091E800877F4B
:103510008093E8006AE270E0CE0101960E942404E4
:103520008091E8008B778093E80010C1C096E7CFC8
:103530008091290590912A05252F332723303105C5
:1035400009F44AC078F52130310509F479C08BE5DA
:1035500090E0EDEFF4E02230310509F0F7C0209162
:10356000E800277F2093E80020912B0530912C055F
:103570008217930708F49C0140E02115310509F0FA
:1035800064C0411162C08091E80082FDC9CF809182
:103590002305882329F2853019F28091E80083FF02
:1035A000F2CFBECF2132310509F43BC022323105C2
:1035B00009F0CCC08330910508F0C8C0FC01EE0FC3
:1035C000FF1FE757FE4F0190F081E02D8A579E4F75
:1035D000DC018C9190E011C0CA019927413089F03B
:1035E00082309105B1F0892B09F0B0C0E4EAF5E032
:1035F000E4918E2F90E0E4EAF5E0009709F4A6C08C
:10360000AECFE2E8F5E0E4918E2F90E0E2E8F5E05D
:10361000F4CFEAE6F5E0E4918E2F90E0EAE6F5E0FB
:10362000ECCF8330910508F091C0880F991FFC0101
:10363000E157FE4F0190F081E02D89E090E08FCFBF
:1036400082E190E0E8E5F5E08ACF809123058823C8
:1036500009F466CF853009F463CF8091E80083FDDB
:103660005FCF8091E80082FD8ECF8091E80080FFDF
:1036700084CF9091F3008091F2002115310519F06B
:103680008830910550F041E0089709F040E08091C2
:10369000E8008E778093E80070CF44914093F1006A
:1036A0003196215031090196E8CF803809F04EC09B
:1036B0008091E800877F8093E800809124058093C3
:1036C000F1009ECE811142C0109127051230F0F515
:1036D0008091E800877F8093E800109324050E9482
:1036E0007803112311F084E005C08091E30087FD89
:1036F000FACF81E08093230542E061EC81E00E94F3
:10370000970342E261EC84E00E94970342E261EC9D
:1037100082E00E94970342E260EC83E00E949703FC
:103720008091230513C080912705813079F481E0D1
:10373000933009F080E0809322051092E900809197
:10374000E800877F8093E8000E9478038091E8007A
:1037500083FF0AC08091E800877F8093E800809112
:10376000EB0080628093EB00AA96E3E00C94E130DA
:103770000E94D7182FEF84E39CE0215080409040B6
:10378000E1F700C0000088E19AE00FB6F894A89530
:10379000809360000FBE90936000FFCF882321F0DC
:1037A0000E943A0E0E949B180895882339F0909148
:1037B000C102892B8093C1020E949B18089588231F
:1037C000D1F19CEF980F913A78F4E2E9F2E091910F
:1037D000891303C0DF0111971C9292E0E839F907C1
:1037E000B1F70E949B18089590E2980F983050F41A
:1037F000877091E001C0990F8A95EAF7892F0E949E
:103800003A0EEFCF9BE5980F933028F490E080E0DC
:103810000E940B05089598E5980F9B3128F490E0DD
:1038200080E00E94E504089593E3980F933118F423
:1038300060E00E940C0F0895CF93C82F8823A9F051
:103840008CEF8C0F813A00F5E2E9F2E0DF018D9117
:10385000C81769F022E0A839B207C9F76C2F80E9D0
:1038600092E00E94CB040E949B18CF910895819111
:10387000C81303C0DF0111971C9232E0E839F30747
:10388000B1F70E949B18EACF80E28C0F883068F471
:10389000C77021E030E001C0220FCA95EAF780919D
:1038A000C102822B8093C102DECF8BE58C0F833067
:1038B00038F42C2F2452330BC9010E940B05D5CFAD
:1038C000E8E5EC0FEB3150F4F0E0EE0FFF1FE55CA4
:1038D000FE4F808191810E94E504C7CF83E38C0F66
:1038E000833118F661E08C2F0E940C0FBECFA8E048
:1038F000B0E0EDE7FCE10C94C5304091D602509168
:10390000D7026091D8027091D9022FB7F8948091B4
:10391000120590911305A0911405B09115052FBFC4
:10392000841B950BA60BB70B11E084369105A105FE
:10393000B10578F10E94FE0BDC01CB010296A11DBE
:10394000B11D89839A83AB83BC83809115019091CB
:10395000160186529D4F20911401422F50E02530D0
:1039600010F044E050E0BE016F5F7F4F0E94A7312E
:1039700082E090E00E944030182F882351F00E948E
:10398000A2046093D6027093D7028093D8029093DA
:10399000D902812F2896E3E00C94E130A9E0B0E051
:1039A000E4EDFCE10C94C53088E0EBE6F5E0DE01E7
:1039B000119601900D928A95E1F7198649E050E041
:1039C00063EE72E0CE0101960E949A319C01409113
:1039D000EC025091ED026091EE027091EF02EFB7B0
:1039E000F8948091120590911305A0911405B0915F
:1039F0001505EFBF841B950BA60BB70B84369105FD
:103A0000A105B10518F411E0232B21F180911D01CE
:103A100090911E0186529D4F20911C01422F50E033
:103A20002A3010F049E050E0BE016F5F7F4F0E94E6
:103A3000A73183E090E00E944030182F882351F096
:103A40000E94A2046093EC027093ED028093EE0258
:103A50009093EF02812F2996E3E00C94E130EF92EE
:103A6000FF921F93CF93DF9300D000D00F92CDB77A
:103A7000DEB77B0190E080E00E944030182F882361
:103A800009F487C080910701482F50E0882311F086
:103A900041E050E0609108017091090166527D4F4C
:103AA000CE0105960E94A7314091D2025091D302D7
:103AB0006091D4027091D5022FB7F89480911205CD
:103AC00090911305A0911405B09115052FBF841B8B
:103AD000950BA60BB70B84369105A105B10540F4F3
:103AE0008BED92E00E9411039D81891709F451C06A
:103AF00081E090E00E94403081111AC010E0809176
:103B0000CE029091CF02A091D002B091D102F701E4
:103B100080839183A283B383812F0F900F900F90A6
:103B20000F900F90DF91CF911F91FF90EF9008952C
:103B300080910F01482F50E0853010F044E050E0B4
:103B4000609110017091110166527D4FCE01019676
:103B50000E94A7318BED92E00E9411039D81891391
:103B6000CDCF0E94A2046093D2027093D3028093BF
:103B7000D4029093D50289819A81AB81BC818093D4
:103B8000CE029093CF02A093D002B093D10211E065
:103B9000B6CF8091DB029091DC02A091DD02B09162
:103BA000DE0289839A83AB83BC831111E4CFA7CF54
:103BB000A0E1B0E0EEEDFDE10C94BC301A82198278
:103BC000FE01339686E0DF011D928A95E9F783E7CF
:103BD000A82E81E0B82E10E000E0EE24E394F12C52
:103BE0002EE7C22E21E0D22EF50181915F018F3F99
:103BF00009F445C0F894E82FE295EF70F0E021A1B8
:103C00008F70A70102C0440F551F8A95E2F7CA01C1
:103C1000922F982B91A392A18095892382A37894C7
:103C200000C0E7E7F1E031E0912C21912F3F09F44A
:103C30009DC0A22FA295AF70B0E090968C9190E0BD
:103C40002F7002C0959587952A95E2F780FD8EC06A
:103C5000832F982A330FCE16DF0639F7F5013197F7
:103C600080818F3F11F00E94E50B50EA5A95F1F7E1
:103C7000E1E0F0E0EC0FFD1FE00FF11F90820F5F1D
:103C80001F4F0430110509F0AFCF48E050E0BE01EE
:103C90006F5F7F4F85EF92E00E949A319C01892BE4
:103CA00049F088E0FE013196A5EFB2E001900D9257
:103CB0008A95E1F70091FE0210E0035F1C4F232B71
:103CC00009F456C081E08093C6020E94BF0490931D
:103CD000C5028093C402F12CE0900905EE2009F49E
:103CE000A1C01A8619861C861B868091F0028A3034
:103CF00008F062C04FE25DE1BE01675F7F4FC8011F
:103D00000E947D10882309F47CC047E75CE1BE0176
:103D1000675F7F4FC8010E947D10882309F471C03E
:103D20004EEC5CE1BE01675F7F4FC8010E947D10D1
:103D3000882309F466C01092F0028091FD0290E0A1
:103D400044E050E0BE01675F7F4F835F9C4F0E945D
:103D50009A3121E02093CD02892B09F044C0E12C57
:103D60008E2D8F296096ECE00C94D83080E071CFD6
:103D7000F090C602FF2009F4AECF8091C40290916A
:103D8000C5020E949304059708F4A5CF44E050E0D3
:103D900065EF72E0C8010E949A31892B59F084E0E6
:103DA000E5EFF2E0D80101900D928A95E1F71092CB
:103DB000C60292CFF12CFBCF8091C7029091C8022E
:103DC0000E949304843F914008F094CF8091CD02EB
:103DD000882329F2FE01399684E0DF011D928A953D
:103DE000E9F71092CD02E091FD02F0E0E35FFC4FB5
:103DF00089859A85AB85BC8580839183A283B383B3
:103E0000AFCF8091F0028F3F31F08F5F8093F0024F
:103E10008A3008F492CF0E94BF049093C802809326
:103E2000C702D4CFF80180819181A281B3818093B0
:103E3000DB029093DC02A093DD02B093DE028BEDF7
:103E400092E00E9411038093DA028090DF0290904A
:103E5000E002A090E102B090E2028091C90290914C
:103E6000CA02A091CB02B091CC0288169906AA068C
:103E7000BB06B1F08092C9029092CA02A092CB0216
:103E8000B092CC020E94A204861A970AA80AB90A24
:103E90008092F1029092F202A092F302B092F402A8
:103EA00088E0E3EEF2E0ABE6B5E001900D928A9592
:103EB000E1F756CF1F93CF93DF93182FEB010E94AA
:103EC0001C1C209739F4812F0E94DF1BDF91CF91BA
:103ED0001F9108958FE99FE00197F1F700C000005E
:103EE0002197EFCFFF920F931F93CF93DF93C62FAE
:103EF000D42F122FFC0185818823A9F060937505CA
:103F00000E94BF049093740580937305C77081E08D
:103F100001C0880FCA95EAF70E94D51BCDB7DEB75E
:103F2000E5E00C94DF3080917505681332C0809114
:103F30007305909174050E949304883C910548F59F
:103F400000E20D0FCD17A9F0C770FF24F3948F2D59
:103F500001C0880FCA95EAF70E94CE1B083048F4CA
:103F60008D2F877001C0FF0C8A95EAF78F2D0E9474
:103F7000D51B70E060E0812F0E945A1F083070F658
:103F8000D77081E001C0880FDA95EAF70E94CE1B56
:103F9000C5CFC77081E001C0880FCA95EAF7F6CF98
:103FA000A8E0B0E0E6EDFFE10C94B8308C01DC0154
:103FB00014968C911497882309F4BEC021E04C918B
:103FC00011965C91119712966C91129713967C91B1
:103FD000139715969C910E9406127C01F801858129
:103FE000882309F447C1C70197578038910508F025
:103FF00072C5FFE0FE1508F48FC08FEF93E00E94BA
:10400000C031811189C059EEA52EBB24B394E110B3
:104010004FC01A821982FE01339686E0DF011D929D
:104020008A95E9F74AE0442E6501BFEFCB1ADB0A17
:10403000C5010E94C03189831A82882309F46CC0AB
:10404000813009F07DC07501E2E0EE0EF11CC60181
:104050000E94C0318A83882309F45EC09FEF980FC5
:104060009330A0F5F3E0AF0EB11CC7010E94C03140
:104070008B83882309F450C01C82DE0111967D01D8
:10408000F7012081222381F2213009F09BC0918128
:104090008281913009F056C0F2E0EF0EF11C70E021
:1040A00060E0893311F460E570E00E945A1F51C04E
:1040B000A11424E0B20681F1C5010E94C031811132
:1040C00001C0EA943FEFA31AB30AA1CF8430D9F418
:1040D00032E0C32ED12CC7012FEFE21AF20A0E9460
:1040E000C031E1E0F0E0EC0FFD1FEC0DFD1D808321
:1040F000882391F08C3749F4E2E0F0E0EC0FFD1FEB
:10410000EC0DFD1D10825701B8CF3FEFC31AD30A43
:1041100087E0C816D104F9F68091B602877061F085
:10412000D80115968C91882339F08091020382FF83
:1041300003C082E00E94E60E2896E0E10C94D430A1
:1041400056019BCF923049F422E0E20EF11C0E940E
:104150001C1C9FEFE91AF90A93CF933031F432E037
:10416000E30EF11C0E94DF1BF4CF943021F08FEF9F
:10417000E81AF80AEECF92E0E90EF11C30E020E0F8
:10418000B7016F5F7F4FD70111964C918053990B08
:104190008A30910560F021153105D9F2EFE9FFE091
:1041A0003197F1F700C0000021503109F4CF429E51
:1041B000F001439EF00D11249C012E0F3F1F842F10
:1041C0007B01DECFE22FF0E0E354FE4F5490822FCC
:1041D00086958695869590E0FC01E355FE4F6490A8
:1041E0002770712C022E02C0759467940A94E2F72E
:1041F000F1E06F227724FC01E356FE4F8490912C6E
:10420000022E02C0959487940A94E2F731E083224B
:104210009924FC01E357FE4FC490D12C02C0D594E1
:10422000C7942A95E2F781E0C822DD246114710465
:1042300019F081EE0E941C1C8114910419F086EE85
:104240000E941C1C70E060E0852D0E945A1F8114A2
:10425000910419F086EE0E94DF1B6114710419F0BD
:1042600081EE0E94DF1BCD2809F473CF70E060E07F
:104270008CE21BCFF701E851FC47E730F10508F06D
:1042800011C4EE56FD4C0C94153126E241EE61EE60
:10429000C8010E94721F40CF27E245EE65EEF8CFBD
:1042A00026E241EE60EEF4CF27E245EE64EEF0CF79
:1042B00026E241EE62EEECCF27E245EE66EEE8CF75
:1042C00028E241E0EBCF80910103816080930103FC
:1042D000609101037091020384E090E00E94FC3140
:1042E0000E94D71819CF809102038860809302033F
:1042F000EFCF809101038260E9CF80910103846058
:10430000E5CF809101038860E1CF80910203816055
:10431000EDCF809102038260E9CF8091010380613B
:10432000D5CF809101038062D1CF80910103806459
:10433000CDCF0E94D718809101038068C7CF8091AC
:1043400001038C60C3CF809102038360CFCF809143
:1043500001038E7FBBCF80910203877FC7CF8091FF
:1043600001038D7FB3CF809101038B7FAFCF80910D
:104370000103877FABCF809102038E7FB7CF8091FF
:1043800002038D7FB3CF809101038F7E9FCF8091F9
:1043900001038F7D9BCF809101038F7B97CF0E947C
:1043A000D718809101038F7791CF80910103837F8C
:1043B0008DCF809102038C7F99CF8091010382FB86
:1043C000992790F921E0922790FB82F990FB83F9DD
:1043D0007DCF80910203982F909591708E7F892BCD
:1043E00090FB81F983CF90910103892F8F7B96FFFA
:1043F00080646CCF0E94D71890910103892F97FB9E
:1044000087F9805863CF61E08EE090E00E94DE3152
:104410005FCF60E0F9CF90910103892F8F7E94FFE9
:10442000806154CF90910103892F8E7F90FF81602E
:104430004DCF90910203892F877F93FF886056CFDD
:1044400085E33BC3A7E7EA16ACE7FA0609F064C3C5
:1044500081E00E94FD0E43E062E081E00E94B90E1F
:104460005BCE8091C1028272F701E052F847E531DC
:10447000F10508F054C0E756FD4C0C9415318091BD
:104480006B0591E0892780936B0510923301809131
:104490003A04816080933A043FCE46E856E063E9EF
:1044A00076E00E94B80538CE43E956E066E876E04B
:1044B000F8CF46E556E061E676E0F3CF41E656E018
:1044C00066E576E0EECF4AE356E068E476E0E9CFD1
:1044D00048E456E06AE376E0E4CF4EE156E06CE271
:1044E00076E0DFCF4CE256E06EE176E0DACF4EEEDA
:1044F00055E06CEF75E0D5CF4CEF55E06EEE75E012
:10450000D0CF61E081E00E946C0606CE61E085E0DC
:10451000FACF61E08DE0F7CF61E082E1F4CFB7E759
:10452000EB16BCE7FB0609F0FFC281E00E94D90E42
:1045300092CFEAE5EE16ECE7FE0609F490C008F02B
:1045400064C021E0E2162CE7F20609F486C033E0ED
:10455000E3163CE7F30609F47AC0E1148CE7F806A9
:1045600009F468C0F8018581C080D180882309F4EE
:104570007AC0C6010E94A511F82E682FC6010E94BC
:10458000800EB6018F2D0E9497110E94220D7C0192
:10459000882ED80115967C9015971696CC90C294CB
:1045A0002FE0C2228091B602877009F1972C772004
:1045B000F9F08F2D807F803469F080E28E0D883095
:1045C000B0F08F2D807E803229F4B1E0BE1578F4F2
:1045D000CC2069F08091020382FF09C082E00E9432
:1045E000E60E8091B6028770992493948111912CE4
:1045F0008F2D82958F70A82EB12C8C3008F09CC026
:10460000F501E255FD4C0C9415319BE5E9169CE74C
:10461000F90639F1ACE5EA16ACE7FA0609F0A2CFE3
:104620008091020382FB882780F991E089270E940C
:10463000841898CF0E94D718BFEFE4E3FCE0B15094
:10464000E040F040E1F700C000000E9482046FEFFC
:104650007FEF90E080E00E94FC310E94B81B81E077
:10466000E6CF80E0E4CFC6010E944C0EF82E89CF41
:10467000EF2DEF70DE2E8F2D807F19F0D29490EF0A
:10468000D9228E2D7720B9F0DD2069F090E29E0DC1
:10469000983010F0E11009C08091C102D82AD09260
:1046A000C1020E949B188E2D45C08091B802D82A65
:1046B000D092B802F6CF0E94DF1BDD20E9F180E244
:1046C0008E0D883010F0811004C08D2D0E943A0E9E
:1046D00006C0D0948091B802D822D092B8020E942D
:1046E0009B182AC0FF2DFF70DF2E8F2D807F803218
:1046F00019F0D29480EFD8228E2D882059F021E035
:10470000821609F47BC0772009F487C0CC2009F415
:1047100049C0C9CF8091020382FD40C07720C1F11A
:10472000DD2039F08091C102D82AD092C1020E94C6
:104730009B1880E00E941C1CE8E0AE1AB108F4E06F
:10474000AF16B10410F40E9431059920B1F08091A8
:10475000B60280FD12C0D80115961C9286958695EA
:1047600086950E94FD0EC8010E94D01F8091B6025E
:104770008695869586950E94D90E20E0F8014081A5
:10478000518162817381848195810E940612D4CC0B
:1047900080E00E94DF1BDD2079F297CF7720A1F027
:1047A000C11004C08D2D0E94D51BC6CF31E0C312AD
:1047B000C3CF8091B7029D2D9823D91609F4BCCFA1
:1047C000D82AD092B702B8CFC110B6CF8D2D0E9493
:1047D000CE1B9091B7028D2D892329F08D2D8095C8
:1047E00089238093B702809199029D2D982309F423
:1047F000A3CFD094D822D09299029ECF772029F0CF
:1048000085E08C1508F498CFCDCF94E09C1508F482
:1048100093CF8D2D0E94CE1B8FCFCC20D1F3893327
:1048200049F4AFEFB7EEE3E0A150B040E040E1F76C
:1048300000C000008E2D0E94DF1B7ECF8F2D86953D
:104840008695837061F0813009F076CFC70193704F
:10485000711002C080E090E00E94E5046DCFC701B6
:104860009370711002C080E090E00E940B0564CF4D
:10487000672D8E2D0E940C0F5FCF8F2D837099F5C1
:1048800071105ACF4E2D429546954770440F440FF4
:104890008E2D8F70042E01C0880F0A94EAF72E2DFA
:1048A0002071E4FE07C02FE030E001C0220F4A95DE
:1048B000EAF720953F2D369536953370323071F0FA
:1048C000333051F04091FF02313029F0822B8423A4
:1048D0000E94090F31CF842B822BFACF282B809195
:1048E000FF028227F5CF8695772011F08F2D8170FA
:1048F000882309F421CF4E2D429546954770440FE9
:10490000440F8E2D8F70042E01C0880F0A94EAF791
:104910002E2D2071E4FE07C02FE030E001C0220FF1
:104920004A95EAF720953F2D36953695337032300B
:1049300071F0333051F040910003313029F0822B77
:1049400084230E94B60EF8CE842B822BFACF282B1C
:10495000809100038227F5CFFF2DFF70FF2E772077
:1049600029F08F2F0E94FD0E8E2D1DCF8E2D0E94BF
:10497000CE1B8F2D0E94D90EDFCE8E2D22EF8216F8
:10498000B1F1281570F030EF8316D1F091EF891650
:1049900091F0772009F45EC0C11085CE8F2D8F7104
:1049A0002AC0A3EF8A1651F1B4EF8B12F2CF809197
:1049B000020382FD2FC08F2D8F717720D9F21BC08B
:1049C000772081F0E4E0EC1508F4B6CE2F2D2F719E
:1049D00081E090E001C0880F2A95EAF790910003EA
:1049E0008927AFCFF5E0FC1508F4A6CEEFCF8F2DC9
:1049F0008F717110BFCF0E94FD0E9ECE80E0772098
:104A000009F49FCF9F2D9F7181E001C0880F9A9577
:104A1000EAF797CF772099F02F2D2F71F22E822F62
:104A20000E94FD0E8091020382FF07C038E0F39ED2
:104A3000C001112483608093B6028F2DDCCF81E00A
:104A40000E94E60E81E08C1508F076CE82E00E948E
:104A5000E60E72CECC2059F0893309F0EBCE9FEFF1
:104A6000A7EEB3E09150A040B040E1F7E1CE8F2D2A
:104A70008F7180CFF6E1EF16FCE7FF0609F0E2CC7C
:104A80008091C1028A7A91E009F490E090939802B3
:104A900069E2811165E380E992E00E94CB040E9403
:104AA0009B183ACB26E1E2162CE7F20609F0D9CCA6
:104AB000809198028111C4CC89E2E2E9F2E028E910
:104AC00032E09191891303C0DF0111971C922E17D8
:104AD0003F07B9F7E4CFF701E851FC47E730F105AC
:104AE00008F4CFCB10927505C7019057839708F053
:104AF000C1CF84E090E00E94C8319093020380937C
:104B00000103F701E150F047E232F10508F0DBCB99
:104B1000E654FD4C0C94153138E7E3163CE7F306F8
:104B200009F007CD82E095CC88E7E8168CE7F80617
:104B300009F018CD82E0FACCCF93DF938091B502D3
:104B4000807F09F04DC08091B402882309F448C0E9
:104B5000E091660550912D05C091B002D091AF0251
:104B60006091B1027091B20247E05E17C9F18E2FD9
:104B700090E0E49FF0011124E25DFA4F24812223AA
:104B800091F1489FF001499FF00D1124DF01A25DD2
:104B9000BA4F11962C9111972C1325C02C912D13DF
:104BA00022C015962C91159721111DC012962D919A
:104BB0003C91261B370B283C3105A8F48091B502A7
:104BC0008F7080618093B502EC5CFA4F80818F70AA
:104BD000806180838FEA92E00E94D01F0E94420E83
:104BE000DF91CF910895FC013196E770BECFADE023
:104BF000B0E0EDEFF5E20C94BC308C0186E0F801FA
:104C0000DE01189601900D928A95E1F7F8018481F2
:104C1000E5809FEAA92E92E0B92E9091B3029111FE
:104C200028C0882319F1EE20F1F0C8010E94DF119D
:104C3000F82E8823C1F087E0F801D50101900D928C
:104C40008A95E1F78091B302813031F48091AF020F
:104C50009091B0020E94D0110E949C258F2D2D961C
:104C6000ECE00C94D830C8010E94D01FFF24F394CC
:104C7000F5CFD080C18082809380F090B4022091E3
:104C8000B1023091B202A401421B530BFF2009F480
:104C9000BCC0483C510508F092C08823F9F29091BD
:104CA000B0028091B502282F207F09F056C0C912AA
:104CB00014C09091AF02D91210C0E11048C08F709B
:104CC00080618093B5028FEA92E00E94D01F8091AC
:104CD000B502F8018683F12CC1CFE11038C06C2DEC
:104CE0008D2D0E94F3026C2D8D2D0E94F302E82E73
:104CF0008111F1CFD886C986888599850E94D01107
:104D0000292F22952F70903458F49F70223088F00C
:104D1000992399F0F8019681907F79F4FE2C9ECF2B
:104D20002A5F2F70223068F0C8010E94D01FEF2C3C
:104D3000F5CF992311F0882389F3805E883070F3D2
:104D4000F3CF803F58F3815F833040F3EDCF809104
:104D5000B50281608093B502BECFC91207C09091A1
:104D6000AF02D91203C0EE2009F470C0C8010E943E
:104D7000DF11882309F477CFEE2009F474CF8091F6
:104D8000B502803288F02091AF023091B0023A83B0
:104D900029839C828B829091B3029D831E828F8394
:104DA000CE0101960E94D01F87E0F801AFEAB2E081
:104DB00001900D928A95E1F70E949C2557CF909122
:104DC000B502292F207F51F48FEA92E00E94D01F74
:104DD00087E0F50111928A95E9F77DCF882309F4E0
:104DE0003DCF8091B0028C11C1CF8091AF02D8121B
:104DF000BDCFE110BBCF9683C8010E94D01F87E0D2
:104E0000F50111928A95E9F729CF483C5105B8F789
:104E1000882309F42BCFFE2CEE2009F424CF8091B7
:104E2000B0028C1120C08091AF02D8121CC08091BA
:104E3000B50280FD0FC0982F907F61F08683903F70
:104E400031F0982F907F905F8F70892B8683C801F7
:104E50000E94D01F87E0F801AFEAB2E001900D9206
:104E60008A95E1F7FBCEC8010E94DF1181119CCF2A
:104E70008091B50281608093B502C8010E94D01F65
:104E8000EDCEABE1B0E0E7E4F7E20C94C4304E8B3A
:104E90005F8B688F798F8A8F192F9B8F911110925A
:104EA000B8021D8A86E0FE017696DE011F9601900B
:104EB0000D928A95E1F70A8D002341F021E04F859C
:104EC000588969897A89C8010E9406120B8B1C8B4C
:104ED00087E0FE013F96DE01189601900D928A95BB
:104EE000E1F7CE0108960E94F72581110CC087E0FA
:104EF000FE013896DE01119601900D928A95E1F738
:104F00004C8541110BC017E08091660590912D05ED
:104F1000891332C06B96E4E00C94E03020912D05AB
:104F200030E0C9010196877099275091660558179E
:104F30001906A1F04D8397E0929FD001939FB00D89
:104F40001124A25DBA4FFE01319601900D929A95FF
:104F5000E1F780932D050E94420ED5CF0E94D7180D
:104F600010922D051092660587E0EFEAF2E0DF016E
:104F70001D928A95E9F7C7CF819FC0011124825DF8
:104F80009A4F0E94F725882329F28091660590E0C8
:104F900001968770992780936605B6CFA6E0B0E0AA
:104FA000E4EDF7E20C94C4300E94BF048C018091C0
:104FB000C2029091C3028017910781F019821A8270
:104FC0000E94BF04682F49815A81792F80E090E0C8
:104FD0000E9441271093C3020093C2022696E4E088
:104FE0000C94E0301F920F920FB60F9211242F9362
:104FF0003F934F935F936F937F938F939F93AF9361
:10500000BF93CF93DF93EF93FF93D091E900DF70CD
:105010008091EC00C82FC17080FDC0E81092E900BB
:105020008091F000877F8093F00078940E94FE18B2
:105030001092E9008091F00088608093F000CD2B01
:10504000CF70C093E900FF91EF91DF91CF91BF91B5
:10505000AF919F918F917F916F915F914F913F9110
:105060002F910F900FBE0F901F9018951F920F92C7
:105070000FB60F9211242F933F934F935F936F932B
:105080007F938F939F93AF93BF93EF93FF93809101
:10509000E10082FF09C08091E20082FF05C080919B
:1050A000E1008B7F8093E1008091DA0080FF24C0D3
:1050B0008091D80080FF20C08091DA008E7F80939D
:1050C000DA008091D90080FF9BC080E189BD82E138
:1050D00089BD09B400FEFDCF81E080932305809156
:1050E0001605811109C00E9428030E94C9038091FE
:1050F000E20084608093E2008091E10080FF17C0AD
:105100008091E20080FF13C08091E2008E7F809347
:10511000E2008091E20080618093E2008091D800FB
:1051200080628093D80019BC85E08093230580912C
:10513000E10084FF29C08091E20084FF25C080E166
:1051400089BD82E189BD09B400FEFDCF8091D80000
:105150008F7D8093D8008091E1008F7E8093E10065
:105160008091E2008F7E8093E2008091E200816076
:105170008093E20080912405882309F447C084E0ED
:1051800080932305809123058091E10083FF27C050
:105190008091E20083FF23C08091E100877F8093AC
:1051A000E10082E080932305109224058091E100C4
:1051B0008E7F8093E1008091E2008E7F8093E200F9
:1051C0008091E20080618093E20042E060E080E054
:1051D0000E9497038091F00088608093F000FF9117
:1051E000EF91BF91AF919F918F917F916F915F915F
:1051F0004F913F912F910F900FBE0F901F901895D8
:1052000019BC109223051092160576CF8091E30009
:1052100087FD02C081E0B4CF83E0B2CF78941F92C3
:105220001FB61F9211248F939F93AF93BF938091CA
:10523000120590911305A0911405B09115050196E2
:10524000A11DB11D8093120590931305A093140521
:10525000B0931505BF91AF919F918F911F901FBE85
:105260001F9018951F921FB61F9211248F939F9322
:10527000AF93BF9380911105811113C080911205E6
:1052800090911305A0911405B09115054196A11DAB
:10529000B11D8093120590931305A0931405B0934C
:1052A0001505BF91AF919F918F911F901FBE1F90C9
:1052B0001895CDB7DEB7AC970FB6F894DEBF0FBE2A
:1052C000CDBF85B7806885BF85B7806885BF84B747
:1052D000877F84BF0FB6F894A8958091600088619D
:1052E00080936000109260000FBE80E890E00FB6DF
:1052F000F89480936100909361000FBE83EE9BE071
:1053000090938F0280938E020E9428030E94C9030B
:105310008091E20084608093E2007894809123057C
:105320008823A1F01091E9001F709091EC00892F63
:10533000817090FD80E8182B1092E9008091E800C0
:1053400083FD0E94FE181F701093E90082E084BD67
:1053500093E095BD9AEF97BD80936E001092F10295
:105360001092F2021092F3021092F4020E944F1176
:10537000811102C00E943F118091D800806180930A
:10538000D8002AE12A95F1F700C08091D900182FA2
:10539000117080FD04C00E94280310922305109311
:1053A000090510930A051093240111110E94532F2F
:1053B000809124018091240194E0811190E09093E8
:1053C000FE0284E0891B8093FD0284E90E94E50BC4
:1053D00086E60E94E50B87E90E94E50B86EC0E94B9
:1053E000E50B07E711E05EE7E52E51E0F52ED80169
:1053F0008D918D018F3F11F00E94E50BE016F106B3
:10540000B1F788E0EDE0F3E0DF01282F1D922A9547
:10541000E9F7E5EFF2E0DF011D928A95E9F790E008
:1054200080E00E94C831863E9E4F21F40E944F11B9
:10543000811168C066EE7EEF90E080E00E94FC3152
:1054400060E082E090E00E94DE3181E08093FF0224
:1054500061E083E090E00E94DE3160E074E184E08E
:1054600090E00E94FC3160E086E090E00E94DE3136
:1054700060E087E090E00E94DE3140E050E0BA0159
:1054800088E090E00E94F03160E084E290E00E94C9
:10549000DE3160E087E190E00E94DE3160E08CE088
:1054A00090E00E94DE3160E08DE090E00E94DE310D
:1054B00019821A821B821C821D821E821F821886FC
:1054C00048E050E068E170E0CE0101960E94CE31E4
:1054D00040E050E0BA0180E290E00E94F03180E0CC
:1054E0000E94B6100E943F1140E050E0BA018FE0E8
:1054F00090E00E94F03140E050E0BA0183E190E09A
:105500000E94F03182E090E00E94C031809303035A
:1055100084E090E00E94C8319093020380930103DD
:105520000E94D81DEFE3FCE93197F1F700C00000BD
:105530000E94D81D80910D0380FF08C06FEF7FEFA0
:1055400090E080E00E94FC310E94820483E090E0C1
:105550000E94C0310E94090F0E94EB0581E08093F8
:105560003A0448E050E068E170E08BE695E00E9484
:10557000B03110923A0480916B058C7FB9F485E3C9
:1055800080936B058091380190913901A0913A0187
:1055900080936C0590936D05A0936E058FE78093C3
:1055A0006F058FEF809370050E942A128091090584
:1055B000811102C00E94562F85E291E090930E0562
:1055C00080930D058091230500E112E1853009F4F7
:1055D000E2C00E94D81DA4E0B3E0BAA3A9A3EDE005
:1055E000F3E0FEA3EDA3DF01E4E0F3E091918D9100
:1055F00023E0EC30F20709F4D8C09817B9F32090F3
:105600000905912C812C10E0ADA1BEA17D90BEA317
:10561000ADA3E9A1FAA15190FAA3E9A3571409F4A3
:1056200076C05724740100E066246394852D86219A
:1056300009F461C0D72CD6202220A1F009831A8357
:105640000E94BF049C838B83F1E0FD8391E0D11025
:1056500001C090E09E8349815A816B817C818D815C
:105660000E944127DD2009F446C080916B058C7FA4
:105670008C3709F040C0F701EB56FE4F80818F3F19
:1056800009F439C0B12CA12C312C90E09C01220FDF
:10569000331FA90143535E4F5AA749A7D901A2530B
:1056A000BE4FBCA7ABA7F701EE5FFB4FF8A7EFA378
:1056B0006501412CF601EB56FE4F80818F3F61F072
:1056C000311287C1041185C1AFA1B8A52C9130E278
:1056D000230F08F42FEF2C934394FFEFCF1ADF0A28
:1056E00027E04212E7CF339437E0A30EB11C48E322
:1056F000A416B104E9F60F5F660C5FEFE51AF50A30
:10570000073009F093CFE9A1FAA1319770821F5FAA
:1057100087E0880E911C183009F076CF0E94FE0BAE
:1057200048C080912305843031F10E9435121092D7
:10573000110528E130E040E40FB6F894A8952093D5
:1057400060000FBE4093600083B7817F846083BF99
:1057500083B7816083BF7894889583B78E7F83BF3A
:105760000FB6F894A89580916000886180936000DE
:10577000109260000FBE80912205882361F00E9484
:10578000D81DEDE0F3E0819181110AC385E193E03A
:105790008E179F07C1F780912305853009F4C1CF8B
:1057A0000E94D7180E94310514CF981328CF0E9469
:1057B000CE270E94351286E0E3E0F5E0DE01119687
:1057C00001900D928A95E1F7D0900405109105059E
:1057D000F0900605E0900705009108051092050578
:1057E000109206051092070510920805812F8F2947
:1057F00009F445C080910105909102050E9493042F
:105800009C018091FC04882309F4EEC22531310506
:10581000B0F18F3F19F08F5F8093FC04112359F092
:105820000E948A059FEF11160CF491E0899F802D4C
:10583000112480930505FF2059F00E948A0591E00C
:105840001F140CF09FEF899F802D11248093060573
:1058500080910505882399F0C0900605CC2079F049
:105860000E94AA05882309F4EFC0809305058C2DBA
:105870000E94AA05882309F4E9C0809306058E2DAD
:10588000802B09F445C08091FF04909100050E948F
:1058900093049C018091FD04882309F4A0C2213562
:1058A0003105B0F18F3F19F08F5F8093FD04EE203A
:1058B00059F00E9468059FEF1E140CF491E0899F37
:1058C000802D112480930705002359F00E9468055C
:1058D00091E010160CF09FEF899F802D112480938A
:1058E000080580910705882399F0C0900805CC2011
:1058F00079F00E94AA05882309F4AAC080930705BD
:105900008C2D0E94AA05882309F4A4C08093080561
:1059100080910405D81219C080910505882311F0E3
:10592000811313C020910605222311F02F110DC001
:1059300090910805992311F0901307C03091070545
:10594000311103C0822B892B11F00E944205DA82AB
:105950001B83FC82ED820E8386E0FE013196A3E07C
:10596000B5E001900D928A95E1F70E943105909182
:105970000C03891721F080930C030E94A2048091EC
:105980002305843009F01ECE83E08093E9008091E6
:10599000E80082FF17CE8091E80090E085FF06C006
:1059A0000E944703882309F457C091E08091E800E2
:1059B0008B778093E800992309F404CE8981EFEF77
:1059C000E80FE33108F073C0F0E0E452FD4C0C94B2
:1059D000153190E0A9A5BAA54C91FC01EE0FFF1F6F
:1059E000E353FE4F2081421B550BEBA5FCA5208104
:1059F000880F991FFC01EB56FE4F81AD281B330B1E
:105A0000449FB001459F700D700D1124229FC0016D
:105A1000239F900D900D1124860F971F0E9420093F
:105A2000382F893208F058CE28E2231B08F420E0F2
:105A3000F601EE5FFB4F213108F020E13081320F9B
:105A400008F43FEF308348CE81E00FCF81E015CFDF
:105A500081E054CF81E05ACF80E2E82EF12C8E0114
:105A60000F5F1F4F8091E80085FD0AC08091E8001C
:105A70008B778093E8000E944703882399F395CFA2
:105A80008091F100D8018D938D01B1E0EB1AF108FE
:105A900049F78BCF1A828CE08B831BC08A818330BD
:105AA00009F140F4813069F0823009F48FC18FEF41
:105AB00089830FC08430D9F71B821C821D821E820D
:105AC00008C00E94A2040E941B316B837C838D83DB
:105AD0009E8340E250E0BE016F5F7F4F82E00E94F4
:105AE000F00F70CD2B81822F90E0FE013496245E62
:105AF0008830910570F7DC01A35FBC4F3C91319376
:105B000001962813F5CFE5CF8A81823059F0853090
:105B100071F680916B0591E0892780936B05109257
:105B20003301D7CF2B813C814D815E8129A33AA3DC
:105B30004BA35CA3CA01B9010E941B3188E290E02B
:105B40000E94DE31C6CF4C816B818A810E94681130
:105B50009827892798279E838D83BBCF2D813E81EF
:105B60003227232732274C816B818A810E94DF10E4
:105B7000B0CF0E940611ADCF9A81933009F097CF34
:105B8000883009F441C0893009F46BC08B818330BF
:105B9000B9F198F48130D1F0823009F09ACF8C813C
:105BA00090916B05292F237081111EC011F0109266
:105BB00033019C7F90936B058CCF843009F089CFA3
:105BC0008C8120E040916E056D810AC04C8122E8F5
:105BD000429F412D112480916C0520E060916D055C
:105BE00090E00E940A0675CF211102C01092330185
:105BF0009C7F916090936B0560E00E946C0669CF7A
:105C00008C8180936F0565CF8B81833039F180F46F
:105C10008130C1F0823009F05CCF80916B05982F04
:105C2000937086958695911101C080E08C8351CF49
:105C3000843009F04ECF80916C058C8380916D0586
:105C40008D8347CF80916E053FEF839FC001112464
:105C500062E870E00E94ED306C833BCF80916F056D
:105C6000E5CF0E942A1235CF80E18A8332CF82E0CD
:105C70008A8387E111CF0A811B8110270127102712
:105C8000AE014F5F5F4F6A01EC80CA018E0D911D1E
:105C90007C01C80187519E4FEC14FD0409F419CF13
:105CA0000731A2E01A0750F40E94C031F601848344
:105CB0000F5F1F4FBFEFCB1ADB0AEBCFD601149655
:105CC0001C92F6CF0A811B81102701271027FE01A5
:105CD00031966F01EC80E00EF12EF11CC801875166
:105CE0009E4F0E151F0509F4F4CE0731F2E01F0791
:105CF00028F4D60114966C910E94DE31BFEFCB1AC6
:105D0000DB0A0F5F1F4FEACF0E94CF10E2CE84E084
:105D1000ACCF0A811B81102701271027FE01319685
:105D20006F01EC809F012E0D311D7901C80189960C
:105D3000CE14DF0409F4CDCE003C31E0130758F453
:105D40000E94C031D60114968C930F5F1F4FFFEF56
:105D5000CF1ADF0AEBCFF6011482F7CF0A811B813D
:105D60001027012710279E012F5F3F4F6901EC800C
:105D7000E00EF12EF11CC80189960E151F0509F4DD
:105D8000A8CE003C31E0130728F4D60114966C919C
:105D90000E94DE31BFEFCB1ADB0A0F5F1F4FEBCF44
:105DA00009BD19BD09B400FEFDCF8091D8008F7DDB
:105DB0008093D8008091E00082608093E000809121
:105DC000E00081FDFCCF0E94D718E5CC88E290E08E
:105DD0000E94C0311B821C821D828E837ACE2B30A2
:105DE000310508F061CD94CD2B30310508F013CD8D
:105DF00046CD8EE14B9B02C08150E1F74B9BFECF1D
:105E000008955B9880E28A95F1F75B9A0895FC010A
:105E10003BE03A95F1F798E020E080E031E040E1A6
:105E20004A95F1F7880F4B9B02C08160232742E01F
:105E30004A95F1F7000040E14A95F1F7915079F762
:105E400090E19A95F1F799B132E03A95F1F70000B7
:105E500040E14A95F1F793FB992790F99227208129
:105E6000920F90830895A1E0B0E0E9E3FFE20C9483
:105E7000C23019828C017C01E60EF11C0E151F0543
:105E800041F481E09981911180E02196E6E00C9443
:105E9000DE300E94F92ECE0101960E94072FF801F4
:105EA00081938F01EBCF539A5B9A089553985B9A35
:105EB000EB9AE9E6F0E080818F738083089561506A
:105EC000770B91E001C0990F6A95EAF720E031E085
:105ED000911108C0222391F05B9A80E28A95F1F734
:105EE0005B980895492F482339F05B9A232740E2B5
:105EF0004A95F1F79695ECCF5B98F9CF5B98EDCF8B
:105F0000FF920F931F93CF93DF93EC018C01060F49
:105F1000111DC017D10729F4CDB7DEB7E5E00C9409
:105F2000DF30F9900E94012F68E08F2D0E945F2FD3
:105F3000F0CF1F920F920FB60F9211240F931F9361
:105F40002F933F934F935F936F937F938F939F9381
:105F5000AF93BF93EF93FF93CF93DF930F92CDB7A0
:105F6000DEB719820E94F92ECE0101960E94072FFA
:105F7000282F082F069506950695982F92959570CF
:105F8000802F8570980F892F837096959695890F2D
:105F9000822787709981892B09F05CC0053008F051
:105FA00059C080E18A95F1F75B9A539A82E08A950D
:105FB000F1F700C05B9888E0089F80011124D801A8
:105FC000AC5FBE4F1696ED91FC9117973097A9F0F4
:105FD000609171017091720114962D913C91159709
:105FE000260F371F11968D919C911297680F791F7C
:105FF00013964C9113978C910995F801EC5FFE4F25
:106000006381662351F02091710130917201848186
:106010009581820F931F0E94802F0E94012F80E1A3
:106020008A95F1F75B9853985B9A80E18A95F1F72E
:10603000F801EC5FFE4F6081662351F02091710101
:106040003091720181819281820F931F0E94332FC0
:106050000E94F92E0F90DF91CF91FF91EF91BF91A8
:10606000AF919F918F917F916F915F914F913F91F0
:106070002F911F910F910F900FBE0F901F901895A9
:106080000F931F93CF93DF93EC0105970CF04CC057
:10609000F894539A5B9885E08A95F1F700008C2F6D
:1060A000869585709C2F9570890F982F9370869593
:1060B000869523E0CC0FDD1F2A95E1F7890F8E012D
:1060C000082B0E94012F00C068E0802F0E945F2FE4
:1060D00080E18A95F1F753985B9A4B9B1EC087E04D
:1060E00090E04B991CC0FE01EC5FFE4F638166237C
:1060F000F9F0209171013091720184819581820FB4
:10610000931F0E94332F811113C0539A5B9A789486
:10611000DF91CF911F910F91089500C0DECF0197BD
:1061200029F4539A5B9A789480E0F2CF00C0D9CFDB
:106130000E94F92E80E28A95F1F75B98539A80E1EC
:106140008A95F1F7CC5FDE4F6881662351F020918C
:1061500071013091720189819A81820F931F0E948F
:10616000802F0E94012F789481E0D2CF2F923F920E
:106170004F925F926F927F928F929F92AF92BF9257
:10618000CF92DF92EF92FF920F931F93CF93DF9303
:10619000CDB7DEB7CA1BDB0B0FB6F894DEBF0FBE60
:1061A000CDBF09942A88398848885F846E847D84AD
:1061B0008C849B84AA84B984C884DF80EE80FD80AF
:1061C0000C811B81AA81B981CE0FD11D0FB6F89425
:1061D000DEBF0FBECDBFED010895AA1BBB1B51E171
:1061E00007C0AA1FBB1FA617B70710F0A61BB70B47
:1061F000881F991F5A95A9F780959095BC01CD01EC
:10620000089597FB072E16F4009407D077FD09D068
:106210000E94ED3007FC05D03EF4909581959F4F8C
:106220000895709561957F4F0895EE0FFF1F0590BB
:10623000F491E02D09946927962769277827872705
:1062400078270895CF92DF92EF92FF92CF93DF935A
:10625000CDB7DEB72A970FB6F894DEBF0FBECDBF1D
:1062600089879A87A985BA852D913D914D915C9139
:1062700029833A834B835C83232B242B252B41F4E6
:1062800024E239ED4BE557E029833A834B835C8365
:1062900069817A818B819C812DE133EF41E050E06F
:1062A0000E94023269017A01A7EAB1E49B01AC01C4
:1062B0000E94213269837A838B839C83ACEEB4EF96
:1062C000A70196010E942F329B01AC0189819A811E
:1062D000AB81BC81820F931FA41FB51FB7FF03C002
:1062E0000197A109B048E985FA8580839183A2834B
:1062F000B3839F772A960FB6F894DEBF0FBECDBF4B
:10630000DF91CF91FF90EF90DF90CF9008950E94A2
:106310002231089580E091E00E9422310895B0E09A
:10632000A0E08093000190930101A0930201B0933B
:1063300003010895FB01DC0104C08D9101908019D7
:1063400021F441505040C8F7881B990B0895FB0178
:10635000DC0102C001900D9241505040D8F70895E1
:10636000DC01CB01FC01F999FECF06C0F2BDE1BD15
:10637000F89A319600B40D9241505040B8F7089504
:10638000F999FECF92BD81BDF89A992780B50895FD
:10639000A8E1B0E042E050E00C94B231DC01A40F7F
:1063A000B51F4150504048F0CB01840F951F2E91EE
:1063B0000E94DF3141505040D0F70895262FF999BF
:1063C000FECF92BD81BDF89A019700B4021639F054
:1063D0001FBA20BD0FB6F894FA9AF99A0FBE089525
:1063E0000396272F0E94DF310E94DE31252F0E9465
:1063F000DF31242F0C94DF310196272F0E94DF31EB
:106400000C94DE31052E97FB1EF400940E94193285
:1064100057FD07D00E94343207FC03D04EF40C9491
:10642000193250954095309521953F4F4F4F5F4F12
:10643000089590958095709561957F4F8F4F9F4FF0
:1064400008950E945632A59F900DB49F900DA49F71
:10645000800D911D11240895B7FF0C9421320E94E4
:106460002132821B930B0895A1E21A2EAA1BBB1B9B
:10647000FD010DC0AA1FBB1FEE1FFF1FA217B30710
:10648000E407F50720F0A21BB30BE40BF50B661F26
:10649000771F881F991F1A9469F7609570958095EA
:1064A00090959B01AC01BD01CF010895A29FB00161
:1064B000B39FC001A39F700D811D1124911DB29F38
:1064C000700D811D1124911D0895F894FFCF96122F
:1064D000A212CC12071342138113C113C613C9139E
:1064E000E413E713EC13EF13F213F513F813FB1394
:1064F000FE130114041407140C140F1412144B147B
:106500008414C614C914CC143C152916E916831733
:10651000DC19041AA61B041AA61B371A581AA61B44
:10652000551B621B5021542145214C2158215C21CF
:1065300060213F224D22542259225E22632268228A
:106540006D22722277227C228122862289228C224D
:106550008C208C208C208C208C208C20382338237D
:10656000722372231E2438249C239C233D24AC24B4
:10657000BD24BD24A7211222AF2179217D21B32181
:106580008121B721C3218D210B229121C721952182
:10659000CB21F3219921CF21FA219F21D521DD2182
:1065A0008521BB218921BF21A321D921E9210322F2
:1065B00009227321AB2119224A2D4E2D842DA32DA2
:1065C000AE2DB92DBC2DBC2DBC2D572D572D342EE5
:0E65D000372E3B2E622E842E872E892EAE2E65
:1065DE0001000000000000010000000000000004A7
:1065EE000100000004050000000000000909000081
:1065FE0000000000017F0439107E0432102B103988
:10660E0005FFFF030100FF0000FF82E200E900EA40
:10661E0000B500B600B700CD008301CC008A019210
:10662E000194012102230224022502260227022AB6
:10663E0002B300B4006F0070009F01CB019F02A057
:10664E0002DA02946697C6F4F5F6F731333200316A
:10665E0031295A1B750A44227B49012701AC000FD0
:10666E0005280548051713120D0C05041614110EF6
:10667E000B0603FF15100F0A0702FFFFFFFF0908A5
:10668E00012E2A2924231C1B2D2B2825221D1AFFFF
:10669E002C2726211E19FFFFFFFF201F186E3F66B5
:1066AE002E6619660455025517552C623F4C3F4411
:1066BE002A441544003305331A332F223622212261
:1066CE000C110F112411390033001E783F802E80DB
:1066DE0019800491029117912C843FA23FA22AA205
:1066EE0015A200B305B31AB32FC436C421C40CD5FA
:1066FE000FD524D539E633E61E0000000000000059
:10670E00000000000000000000000000000000007B
:10671E00000000000000000000000000000404045F
:10672E00040404040404040404040404010404041E
:10673E000404040404040401040104040404040411
:10674E000404040401080108080108000000000008
:0E675E0000000000000000000000000000002D
:00000001FF
